:020000040000FA
:06000000AFEF3DF012001D
:060008001DEF17F01200CD
:06002A000500B37B00009D
:10003000E002000004000000AF7B0000FB010000B4
:1000400004000000A77B0000D202000008000000AE
:10005000A57B0000E402000002000000907B00008D
:080060008E02000015000000F3
:0C0104000401006B0051006E016A015004
:10011000000AE8AE02D0D89004D0040E005C000EB5
:10012000015855E20051260DF3CF01F4F4CF02F44B
:10013000000E0127010E022301C4E9FF02C4EAFFF9
:10014000EF6A01C4E9FF02C4EAFF250EE926000EAA
:10015000EA22EF9001C4E9FF02C4EAFF250EE92676
:10016000000EEA22EF8201C4E9FF02C4EAFF250E75
:10017000E926000EEA22EF8401C4E9FF02C4EAFF87
:10018000250EE926000EEA22EF9801C4E9FF02C419
:10019000EAFF250EE926000EEA22EF9601C4E9FFE8
:1001A00002C4EAFF0F0EE926000EEA22EF6801C43E
:1001B000E9FF02C4EAFF210EE926000EEA22700ED2
:1001C000EE6E170EEE6EEE6AEE6A002B9DD7010101
:1001D000986B040E996F9A6B9B6B9C6B9D6B1200D6
:1001E0000401006B0051006E016A0150000AE8AE84
:1001F00002D0D89004D0040E005C000E015863E2D7
:100200000051260DF3CF01F4F4CF02F4000E0127C4
:10021000010E022301C4E9FF02C4EAFFEF50006EA1
:10022000016A00BE0168005001104BE101C4E9FF02
:1002300002C4EAFF010EEF6E01C4E9FF02C4EAFF47
:100240000B0E9EC1EBFF0C0E9FC1EBFF01C4E9FF3B
:1002500002C4EAFF0D0EEB6A0E0EEB6A01C4E9FF61
:1002600002C4EAFFEE52060EE926000EEA22EE6A0A
:10027000EE6AEE6AEE6A01C4E9FF02C4EAFF250EE7
:10028000E926000EEA22EF8001C4E9FF02C4EAFF7A
:10029000250EE926000EEA22EF9601C4E9FF02C40A
:1002A000EAFF0F0EE926000EEA22EF6801C4E9FF1B
:1002B00002C4EAFF250EE926000EEA22EF82005171
:1002C00004D0002B8FD7FE0E00D012000101A051E8
:1002D000260DF3CFE9FFF4CFEAFF000EE926010E69
:1002E000EA22EFCF02F0036A02BE0368040E02188E
:1002F00001E1035002E0000E01D0010E006E016A20
:10030000005000D012000101A151260DF3CFABF433
:10031000F4CFACF4000E0401AB27010EAC23ABC448
:10032000E9FFACC4EAFFEF50006E016A00BE01684D
:10033000040E001801E1015007E0ABC4CEF1ACC4DB
:10034000CFF18FEC0BF063D00101A1510101A66F39
:10035000EAD90101C46BC56B0101C3690101110E2A
:10036000C26FABC4E9FFACC4EAFF180EE926000E69
:10037000EA22EECFBEF1EECFBFF1EECFC0F1EFCF6C
:10038000C1F1ABC4E9FFACC4EAFF140EE926000ECC
:10039000EA22EECFBAF1EECFBBF1EECFBCF1EFCF58
:1003A000BDF1ABC4E9FFACC4EAFF0D0EE926000EB7
:1003B000EA22EECFB8F1EDCFB9F1ABC4E9FFACC49E
:1003C000EAFF0B0EE926000EEA22EECFB6F1EDCFE2
:1003D000B7F1ABC4E9FFACC4EAFFEE52E9CFB4F128
:1003E000EACFB5F1DEEC07F0ABC4E9FFACC4EAFF3D
:1003F000140EE926000EEA22EE2AEE22EE22EE226A
:10040000ABC4E9FFACC4EAFF050EEF6E00D01200EA
:100410000101A251260DF3CFAFF4F4CFB0F4000EDA
:100420000401AF27010EB023AFC4E9FFB0C4EAFF57
:100430000F0EEB50006E016AFF0E001801E1015033
:1004400002E1000EBBD0AFC4E9FFB0C4EAFF250E45
:10045000E926000EEA22EF50020B01E0010E006EC9
:10046000016A0050011002E1000EA8D0AFC4E9FFFC
:10047000B0C4EAFF100EE926000EEA22EECFC4F166
:10048000EDCFC5F1AFC4E9FFB0C4EAFF0F0EEB50EA
:100490000101C36F0101100EC26FAFC4E9FFB0C408
:1004A000EAFF180EE926000EEA22EECFBEF1EECFEB
:1004B000BFF1EECFC0F1EFCFC1F1AFC4E9FFB0C4DF
:1004C000EAFF140EE926000EEA22EECFBAF1EECFD3
:1004D000BBF1EECFBCF1EFCFBDF1AFC4E9FFB0C4CB
:1004E000EAFF0D0EE926000EEA22EECFB8F1EDCFBD
:1004F000B9F1AFC4E9FFB0C4EAFF0B0EE926000E64
:10050000EA22EECFB6F1EDCFB7F1AFC4E9FFB0C448
:10051000EAFFEE52E9CFB4F1EACFB5F1DEEC07F035
:10052000AFC4E9FFB0C4EAFF100EE926000EEA22CC
:10053000EECF00F0EFCF01F0026A036AAFC4E9FF2B
:10054000B0C4EAFF140EE926000EEA220050EE269F
:100550000150EE220250EE220350EE22AFC4E9FF1A
:10056000B0C4EAFF250EE926000EEA22EF92AFC4DE
:10057000E9FFB0C4EAFF250EE926000EEA22EF9853
:10058000AFC4E9FFB0C4EAFF0F0EEB500101E66F04
:100590007FEC24F0AFC4E9FFB0C4EAFF0F0EE926F8
:1005A000000EEA22EF68AFC4E9FFB0C4EAFF250EEF
:1005B000E926000EEA22EF82010E00D012000101AE
:1005C000A351260DF3CFE9FFF4CFEAFF000EE92691
:1005D000010EEA220F0EE926000EEA22EF50006E0D
:1005E000016AFF0E001801E1015004E184EC23F0E0
:1005F00014D013D0A351260DF3CFE9FFF4CFEAFFB7
:10060000000EE926010EEA22250EE926000EEA2256
:10061000EF50020B01E0010E00D012000101A451C5
:10062000260DF3CFADF4F4CFAEF4000E0401AD27E8
:10063000010EAE23ADC4E9FFAEC4EAFF0F0EEB50CE
:10064000006E016AFF0E001801E101502EE1010168
:10065000DB51E66EADC4E9FFAEC4EAFF0F0EE9263A
:10066000000EEA22E552E750EF6EADC4E9FFAEC4DA
:10067000EAFF0F0EEB500101E56F71EC24F0ADC401
:10068000E9FFAEC4EAFF100EEB6A110EEB6A280E0A
:100690000101F96FFA6BADC4E9FFAEC4EAFF0F0EBA
:1006A000EB500101F86F49EC27F0ADC4E9FFAEC48F
:1006B000EAFF100EE926000EEA22EECFABF4EDCFF2
:1006C000ACF40401CA0EAB5D030EAC5902E3000E9C
:1006D00029D0ADC4E9FFAEC4EAFF250EE926000E1D
:1006E000EA22EF880101A5510101DC6F94EC23F0AF
:1006F0000401AB2B000EAC23ADC4E9FFAEC4EAFF8E
:10070000100EABC4EBFF110EACC4EBFFCA0EAB5D19
:10071000030EAC5905E30101A4510101A26F78DE7B
:10072000010E00D012000101A651260DF3CF65F491
:10073000F4CF66F4000E04016527010E662365C43C
:10074000E9FF66C4EAFF250EE926000EEA22EF5013
:10075000080B01E0010E006E016A0050011002E179
:10076000000E0DD090EC24F065C4E9FF66C4EAFFEA
:10077000250EE926000EEA22EF96010E00D01200A7
:100780000101A751260DF3CF00F4F4CF01F4000EC0
:1007900004010027010E012300C4E9FF01C4EAFFA0
:1007A000250EE926000EEA22EF50080B01E0010EAB
:1007B000006E016A0050011035E000C4E9FF01C479
:1007C000EAFF250EE926000EEA22EF50040B01E0B5
:1007D000010E006E016A005001100FE0280E0101A9
:1007E000F66FF76B35EC27F000C4E9FF01C4EAFFB0
:1007F000250EE926000EEA22EF9400C4E9FF01C4A9
:10080000EAFF250EE926000EEA22EF88AAC1E3F1ED
:10081000ABC1E4F1A8C1E1F1A9C1E2F12CEC24F0F3
:1008200008D007D0006A016A00C0F3FF01C0F4FFDE
:1008300000D012000101AC51260DF3CF65F4F4CFC6
:1008400066F4000E04016527010E662365C4E9FF06
:1008500066C4EAFF250EE926000EEA22EF50080BD7
:1008600001E0010E006E016A005001104AE065C40B
:10087000E9FF66C4EAFF250EE926000EEA22EF50E2
:10088000040B01E0010E006E016A005001100FE040
:10089000280E0101F66FF76B35EC27F065C4E9FF10
:1008A00066C4EAFF250EE926000EEA22EF9465C42D
:1008B000E9FF66C4EAFF120EE926000EEA22EE50B6
:1008C000ED100CE190EC24F065C4E9FF66C4EAFF8A
:1008D000250EE926000EEA22EF9615D065C4E9FF41
:1008E00066C4EAFF120EE926000EEA22EE06EF5A6F
:1008F00013EC24F0ADC1E9FFAEC1EAFFEF6E010ECB
:1009000002D0000E00D012000101AF51260DF3CF2E
:10091000E9FFF4CFEAFF000EE926010EEA22250ED8
:10092000E926000EEA22EF50080B01E0010E00D08C
:10093000120004010F6B006B0051006E016A015040
:10094000000AE8AE02D0D89004D0040E005C000E7D
:10095000015801E3F0D10051260DF3CF09F4F4CF93
:100960000AF4000E0927010E0A2309C4E9FF0AC48C
:10097000EAFF250EE926000EEA22EF50080B01E0FF
:10098000010E026E036A0250031013E109C4E9FF6D
:100990000AC4EAFF250EE926000EEA22EF50100BEA
:1009A00001E0010E046E056A0450051002E1000E1C
:1009B00001D0010E006E016A0050011001E0B8D1B3
:1009C00009C4E9FF0AC4EAFFEF50026E036A02BEDF
:1009D00003680250031029E009C4E9FF0AC4EAFFD2
:1009E000EF50066E076A06BE0768010E061801E1A1
:1009F000075011E109C4E9FF0AC4EAFF250EE92600
:100A0000000EEA22EF50010B086E096A010E081869
:100A100001E1095002E0000E01D0010E046E056AEA
:100A20000450051002E1000E01D0010E006E016AB3
:100A30000050011001E07CD17AEC3DF01AC005F4C1
:100A40001BC006F41CC007F41DC008F409C4E9FF6C
:100A50000AC4EAFF1D0EE926000EEA22EE50040148
:100A6000055D016FEE500659026FEE500759036F96
:100A7000EE500859046F09C4E9FF0AC4EAFF210EC9
:100A8000E926000EEA220151EE5C0251EE580351B4
:100A9000EE580451EE5801E34BD184EC23F00009E9
:100AA00001E149D17AEC3DF01AC000F01BC001F021
:100AB0001CC002F01DC003F009C4E9FF0AC4EAFF2C
:100AC0001D0EE926000EEA2200C0EEFF01C0EEFF77
:100AD00002C0EEFF03C0EEFF09C4E9FF0AC4EAFF4B
:100AE000210EE926000EEA22EE2AEE22EE22EE2266
:100AF00009C4E9FF0AC4EAFF1C0EE926000EEA2237
:100B0000EF2A09C4E9FF0AC4EAFFEF50006E016A48
:100B100000BE0168060E001801E101506AE0070EF0
:100B2000001801E1015065E0050E001801E10150D7
:100B300041E00A0E001801E101503CE0040E0018EB
:100B400001E101502DE0020E001801E101500AE020
:100B5000030E001801E1015001E06AD00401020E09
:100B60000F6F66D009C4E9FF0AC4EAFF1C0EEB5000
:100B7000006E016A0150000AE8AE02D0D89004D09D
:100B8000030E005C000E015804E20401120E0F6F08
:100B900006D009C4CEF10AC4CFF18FEC0BF048D0D7
:100BA0000401110E0F6F09C4E9FF0AC4EAFF050E24
:100BB000EF6E3ED009C4E9FF0AC4EAFF1C0EEB50F9
:100BC000006E016A0150000AE8AE02D0013405D07F
:100BD000030ED8800054000E015407E209C4CEF180
:100BE0000AC4CFF18FEC0BF003D00401010E0F6F9C
:100BF0001FD009C4E9FF0AC4EAFF1C0EEB50006EC7
:100C0000016A0150000AE8AE02D0013405D0030E9B
:100C1000D8800054000E015407E209C4CEF10AC482
:100C2000CFF18FEC0BF003D00401100E0F6F00D04A
:100C300004010F51006E016A0150000AE8AE02D0B3
:100C4000013405D0000ED8800054000E015470E22B
:100C50000F51006E016A100E001801E1015015E0FD
:100C600009C4E9FF0AC4EAFF140EE926000EEA22CD
:100C7000EFCF0BF4EE2AEFCF0CF4EE22EFCF0DF412
:100C8000EE22EFCF0EF4EF2210D009C4E9FF0AC420
:100C9000EAFF140EE926000EEA22EECF0BF4EECFA7
:100CA0000CF4EECF0DF4EFCF0EF40101C46BC56B65
:100CB0000101C36904010F510101C26F09C4E9FFB9
:100CC0000AC4EAFF180EE926000EEA22EECFBEF1B2
:100CD000EECFBFF1EECFC0F1EFCFC1F10BC4BAF14F
:100CE0000CC4BBF10DC4BCF10EC4BDF109C4E9FFD5
:100CF0000AC4EAFF0D0EE926000EEA22EECFB8F193
:100D0000EDCFB9F109C4E9FF0AC4EAFF0B0EE926E9
:100D1000000EEA22EECFB6F1EDCFB7F109C4E9FF3C
:100D20000AC4EAFFEE52E9CFB4F1EACFB5F146D9F1
:100D30000401002B01D61200140E0101E36FE46BD5
:100D40000101000EE16F040EE26F2CEC24F00101B2
:100D5000000ECC6F040ECD6FB4EC0AF0B0C1E9FF09
:100D6000B1C1EAFF060EE926000EEA22EECF14F426
:100D7000EECF15F4EECF16F4EFCF17F4000180514B
:100D80000401186F000181510401196F00018251A3
:100D900004011A6F0001835104011B6F1C6B060EC6
:100DA0001D6FB2C11EF4B3C11FF41EC4C8F21FC42C
:100DB000C9F2FFEC37F0F3CF1EF4F4CF1FF40C0EA2
:100DC0000201D06FD16B0201140ECE6F040ECF6FF3
:100DD0007EEC38F0F3CF21F4F4CF22F40401211F8C
:100DE000221F240E0101F66FF76B35EC27F004018A
:100DF00021510101DC6F94EC23F004012251010127
:100E0000DC6F94EC23F0140E0101F66FF76B35ECF8
:100E100027F0B2C1C6F1B3C1C7F1FBD9F3CF21F4BA
:100E2000F4CF22F404011051211902E111512219C9
:100E300004E090EC24F0010EC0D00C51F00BE8421D
:100E4000E842E842E842006E016AD8900036013676
:100E5000D89000360136140E005E000E015A00C014
:100E600023F42351006E016A00500101B25DB26F9C
:100E70000150B359B36F140EB25F000EB35B04019F
:100E80000C51F00BE842E842E842E8420101F66FFB
:100E9000F76BD890F637F737D890F637F737140E48
:100EA000F627000EF72335EC27F0B0C1CAF1B1C127
:100EB000CBF10101000EC86F040EC96F18DA0401EE
:100EC000206F2051006E016A0150000AE8AE02D086
:100ED000D89004D0FE0E005C000E015814E2B2C19E
:100EE000D5F1B3C1D6F10101000ED36F040ED46F5A
:100EF000B0C1D1F1B1C1D2F1040120510101D06FD3
:100F00001DEC0CF058D090EC24F004012051006E40
:100F1000016AFF0E001801E101504DE10101B251DB
:100F2000040108270101B35104010923000E0A231B
:100F30000B230D51020B01E0010E026E036A0250F9
:100F4000031009E10D51010B046E056A04500510F0
:100F500002E1000E01D0010E006E016A0050011086
:100F600005E0082B000E09230A230B230101C46BA3
:100F7000C56B0101C3690101040EC26F04C4BEF157
:100F800005C4BFF106C4C0F107C4C1F108C4BAF179
:100F900009C4BBF10AC4BCF10BC4BDF100C4B8F173
:100FA00001C4B9F102C4B6F103C4B7F1B0C1B4F1E0
:100FB000B1C1B5F103D8010E00D0120084EC23F0CA
:100FC000000901E1FBD7B6C167F4B7C168F4B8C145
:100FD00069F4B9C16AF4BAC16BF4BBC16CF4BCC1A9
:100FE0006DF4BDC16EF4BEC16FF4BFC170F4C0C179
:100FF00071F4C1C172F40401749D749F7391739371
:10100000739573970101C2510401746FBAEC24F017
:10101000F3CF75F4F4CF76F40401000E755D040E81
:10102000765904E3756B040E766F0DD0360ED880BA
:101030007555000E765505E2360E755F000E765B2F
:1010400002D0756B766B776B786B796B7A6B01017D
:10105000670ECC6F040ECD6F87DA140E0101C42722
:10106000000EC523C251006E016A0050020B10E051
:10107000040EC427000EC5230401020E7B6F040E6C
:101080007C6F7D6F7E6B7399738B738D739F05D0AF
:1010900004017389739B738D739F00018051040158
:1010A0007F6F000181510401806F000182510401B2
:1010B000816F000183510401826FB4C1E9FFB5C1A2
:1010C000EAFF060EE926000EEA22EECF83F4EECF09
:1010D00084F4EECF85F4EFCF86F4876B060E886F2D
:1010E000C4C189F4C5C18AF489C4C8F28AC4C9F2EA
:1010F000FFEC37F0F3CF89F4F4CF8AF40C0E020141
:10110000D06FD16B02017F0ECE6F040ECF6F7EECDD
:1011100038F0F3CF77F4F4CF78F40401771F781F19
:1011200077C465F478C466F40101C351006E016AA6
:10113000FF0E001801E1015004E10101DB51010142
:10114000C36F140E0101F96FFA6B0101C351010164
:10115000F86F49EC27F0C4C1AEF2C5C1AFF202018D
:10116000060EAD6FB4C1ABF2B5C1ACF255EC32F0C6
:10117000140E0101DF6FE06B0101670EDD6F040EDD
:10118000DE6FB0EC23F00101C251006E016A005025
:10119000020B0BE0040E0101DF6FE06B01017B0E1F
:1011A000DD6F040EDE6FB0EC23F0140E0101F96F59
:1011B000FA6B0101C3510101F86F49EC27F0C4C17A
:1011C000C6F1C5C1C7F125D8F3CF65F4F4CF66F4F5
:1011D000240E0101F96FFA6B0101C3510101F86F8F
:1011E00049EC27F0040166510101DC6F94EC23F017
:1011F000040165510101DC6F94EC23F00101F96BEE
:10120000FA6B0101C3510101F86F49EC27F0A0EF1F
:1012100026F00401010E8B6F8C6B8D6B0101C6C132
:1012200000F0C7C101F0C607000EC75B00500110F7
:101230004DE013EC24F004018E6F8BC400F0016AC2
:1012400000BE01680050011019E18C518E258C6F91
:10125000006E016A8E51000101AF02D0D89003D018
:10126000005D000E015909E204018D2B8D51006EC5
:10127000016A0050011001E18C2B18D08D518E2590
:101280008D6F006E016A8E51000101AF02D0D890BF
:1012900003D0005D000E015909E204018C2B8C5132
:1012A000006E016A0050011001E18D2B8BC402F029
:1012B000036A02BE03680250031002E0000E01D070
:1012C000010E006E016A00C08BF4A8D704018D5195
:1012D000006E016A001C8D6F8C51006E016A001C4B
:1012E0008C6F8CC4F3FF8DC4F4FF00D01200040196
:1012F000FE0E276F266B2651006E016A0150000A10
:10130000E8AE02D0D89004D0040E005C000E015864
:1013100001E394D02651260DF3CF24F4F4CF25F425
:10132000000E2427010E252324C4E9FF25C4EAFF6B
:10133000EF50006E016A00BE01680050011001E12B
:101340007AD024C4E9FF25C4EAFF0B0EE926000E7B
:10135000EA22EECF00F0EFCF01F0C8C1E9FFC9C12A
:10136000EAFF020EE926000EEA22EECF02F0EFCFEE
:1013700003F00250001802E1035001185CE124C49C
:10138000E9FF25C4EAFFEF50006E016A00BE016864
:10139000010E001801E1015002E12651276F24C41B
:1013A000E9FF25C4EAFF0D0EE926000EEA22EECF82
:1013B00002F0EFCF03F0C8C1E9FFC9C1EAFFEECFE9
:1013C00004F0EFCF05F00450021802E105500318B5
:1013D00027E1CAC1E9FFCBC1EAFF060EE926000EEC
:1013E000EA22EECF06F0EECF07F0EECF08F0EFCF17
:1013F00009F024C4E9FF25C4EAFFEE52060EE926EF
:10140000000EEA22EE500001061909E1EE5007191C
:1014100006E1EE50081903E1EE50091900E102E07F
:10142000000E01D0010E006E016A0050011003E0B1
:101430000401265198D00401262B5DD72751260D93
:10144000F3CF24F4F4CF25F4000E2427010E252336
:101450002751026E036AFE0E021801E103500EE0EE
:1014600024C4E9FF25C4EAFFEF50046E056A04BEF8
:101470000568010E041801E1055002E0000E01D0DC
:10148000010E006E016A0050011060E00A0EE66E67
:10149000E66ACAC1E6FFCBC1E6FF24C4E9FF25C462
:1014A000EAFFEE52E9CF00F0EACF01F000C0E6FF1C
:1014B00001C0E6FF28EC3BF0F56E060EE15EF5504C
:1014C000C8C1E9FFC9C1EAFF020EE926000EEA22FF
:1014D000EECF00F0EFCF01F024C4E9FF25C4EAFF0E
:1014E0000B0E00C0EBFF0C0E01C0EBFFC8C1E9FF03
:1014F000C9C1EAFFEECF00F0EFCF01F024C4E9FF4D
:1015000025C4EAFF0D0E00C0EBFF0E0E01C0EBFF7D
:1015100024C4E9FF25C4EAFF250EE926000EEA22CD
:10152000EF9624C4E9FF25C4EAFF0F0EE926000E5A
:10153000EA22EF6824C4E9FF25C4EAFF250EE92664
:10154000000EEA22EF82040127510DD02751006ED0
:10155000016AFE0E001801E1015003E1FF0E03D005
:1015600002D0FE0E00D01200CCC1E9FFCDC1EAFFCF
:10157000EECFC8F2EDCFC9F2FFEC37F0F3CF00F0B9
:10158000F4CF01F0CCC1E9FFCDC1EAFF00C0EEFF0E
:1015900001C0EDFFCCC1E9FFCDC1EAFF020EE92693
:1015A000000EEA22EECFC8F2EDCFC9F2FFEC37F021
:1015B000F3CF00F0F4CF01F0CCC1E9FFCDC1EAFFD9
:1015C000020E00C0EBFF030E01C0EBFFCCC1E9FF30
:1015D000CDC1EAFF040EE926000EEA22EECFCAF2E0
:1015E000EECFCBF2EECFCCF2EFCFCDF210EC38F065
:1015F0001AC000F01BC001F01CC002F01DC003F0B7
:10160000CCC1E9FFCDC1EAFF040EE926000EEA22B3
:1016100000C0EEFF01C0EEFF02C0EEFF03C0EEFF10
:10162000CCC1E9FFCDC1EAFF080EE926000EEA228F
:10163000EECFCAF2EECFCBF2EECFCCF2EFCFCDF2BF
:1016400010EC38F01AC000F01BC001F01CC002F012
:101650001DC003F0CCC1E9FFCDC1EAFF080EE926A9
:10166000000EEA2200C0EEFF01C0EEFF02C0EEFF56
:1016700003C0EEFFCCC1E9FFCDC1EAFF0E0EE926A3
:10168000000EEA22EECFC8F2EDCFC9F2FFEC37F040
:10169000F3CF00F0F4CF01F0CCC1E9FFCDC1EAFFF8
:1016A0000E0E00C0EBFF0F0E01C0EBFFCCC1E9FF37
:1016B000CDC1EAFF100EE926000EEA22EECFC8F2F5
:1016C000EDCFC9F2FFEC37F0F3CF00F0F4CF01F02B
:1016D000CCC1E9FFCDC1EAFF100E00C0EBFF110E37
:1016E00001C0EBFFCCC1E9FFCDC1EAFF120EE92634
:1016F000000EEA22EECFC8F2EDCFC9F2FFEC37F0D0
:10170000F3CF00F0F4CF01F0CCC1E9FFCDC1EAFF87
:10171000120E00C0EBFF130E01C0EBFF1200CEC192
:10172000E9FFCFC1EAFF0F0EEB50006E016AFF0E1A
:10173000001801E101501CE0CEC1E9FFCFC1EAFF72
:101740000F0EEB500101E66F7FEC24F0CEC1E9FFF4
:10175000CFC1EAFF0F0EE926000EEA22EF68CEC1E4
:10176000E9FFCFC1EAFF250EE926000EEA22EF824B
:10177000CEC1E9FFCFC1EAFFEE52060EE926000E08
:10178000EA22EE6AEE6AEE6AEE6ACEC1E9FFCFC1E6
:10179000EAFF0D0EEB6A0E0EEB6ACEC1E9FFCFC178
:1017A000EAFF250EE926000EEA22EF50080B01E0C1
:1017B000010E006E016A0050011002E090EC24F06E
:1017C000CEC1E9FFCFC1EAFF250EE926000EEA22CD
:1017D000EF96CEC1E9FFCFC1EAFF210EE926000E48
:1017E000EA22700EEE6E170EEE6EEE6AEE6ACEC153
:1017F000E9FFCFC1EAFF250EE926000EEA22EF98A5
:10180000CEC1E9FFCFC1EAFF250EE926000EEA228C
:10181000EF50010B006E016A0050011007E0CEC1CD
:10182000E9FFCFC1EAFF010EEF6E05D0CEC1E9FF9F
:10183000CFC1EAFFEF6A00D012000401366B01014C
:10184000D051260DF3CF34F4F4CF35F4000E04015B
:101850003427010E352334C4E9FF35C4EAFF180EDE
:10186000E926000EEA22EECF2CF4EECF2DF4EECFD7
:101870002EF4EFCF2FF434C4E9FF35C4EAFF140E81
:10188000E926000EEA22EECF30F4EECF31F4EECFAF
:1018900032F4EFCF33F4D3C1E9FFD4C1EAFF040E31
:1018A000E926000EEA22EECF24F4EECF25F4EECFA7
:1018B00026F4EFCF27F40101D551040124270101BB
:1018C000D65104012523000E2623272334C4E9FF23
:1018D00035C4EAFF140EE926000EEA22EECF28F402
:1018E000EECF29F4EECF2AF4EFCF2BF434C4E9FF86
:1018F00035C4EAFF1C0EE926000EEA22EF6A7AECF4
:101900003DF01AC000F01BC001F01CC002F01DC069
:1019100003F034C4E9FF35C4EAFF1D0EE926000ECA
:10192000EA2200C0EEFF01C0EEFF02C0EEFF03C0DE
:10193000EEFF34C4E9FF35C4EAFF210EE926000EAC
:10194000EA22700EEE6E170EEE6EEE6AEE6A34C488
:10195000E9FF35C4EAFFEF50006E016A00BE01687E
:10196000010E001801E1015001E0B7D090EC24F025
:1019700001019A2B000E9B239C239D2334C4E9FF75
:1019800035C4EAFF140EE926000EEA229AC1EEFFE2
:101990009BC1EEFF9CC1EEFF9DC1EEFF0401242B15
:1019A00025232623272334C4E9FF35C4EAFF180E74
:1019B000E926000EEA2224C4EEFF25C4EEFF26C469
:1019C000EEFF27C4EEFF34C4E9FF35C4EAFF140E6E
:1019D000E926000EEA22EECF28F4EECF29F4EECF6E
:1019E0002AF4EFCF2BF434C4E9FF35C4EAFF140E18
:1019F000E926000EEA22EE2AEE22EE22EE22D3C1E2
:101A0000E9FFD4C1EAFF0D0EE926000EEA22EF50ED
:101A1000020B01E0010E006E016A0050011036E079
:101A20000A0EE66EE66AD1C1E6FFD2C1E6FF34C413
:101A3000E9FF35C4EAFFEE52E9CF00F0EACF01F04A
:101A400000C0E6FF01C0E6FF28EC3BF0F56E060E95
:101A5000E15EF550D3C1E9FFD4C1EAFFEECF00F05B
:101A6000EFCF01F034C4E9FF35C4EAFF0D0E00C02A
:101A7000EBFF0E0E01C0EBFF0401120E366F34C4F3
:101A8000E9FF35C4EAFF020EEF6E26D0040E366F72
:101A900024C428F425C429F426C42AF427C42BF42A
:101AA000D3C1E9FFD4C1EAFFE926000EEA22EECF56
:101AB00024F4EECF25F4EECF26F4EFCF27F434C490
:101AC000E9FF35C4EAFFEE52060EE926000EEA22CF
:101AD000EE6AEE6AEE6AEE6A11D3D3C1E9FFD4C1B1
:101AE000EAFF0D0EE926000EEA22EF50040B01E09A
:101AF000010E006E016A0050011009E090EC24F024
:101B000034C4CEF135C4CFF10ADE3BD3F7D2D3C112
:101B1000E9FFD4C1EAFF080EE926000EEA2204011B
:101B20002851EE1809E12951EE1806E12A51EE1864
:101B300003E12B51EE1800E101E0DED234C4E9FFED
:101B400035C4EAFFEF50006E016A00BE0168020E64
:101B5000001801E1015074E1D3C1E9FFD4C1EAFFEB
:101B60000D0EE926000EEA22EF50100B01E0010EE7
:101B7000006E016A0050011060E034C4E9FF35C412
:101B8000EAFF180EE926000EEA2224C4EEFF25C45F
:101B9000EEFF26C4EEFF27C4EEFF34C4E9FF35C4D0
:101BA000EAFF1C0EE926000EEA22EF6A7AEC3DF00D
:101BB0001AC000F01BC001F01CC002F01DC003F0F1
:101BC00034C4E9FF35C4EAFF1D0EE926000EEA22FF
:101BD00000C0EEFF01C0EEFF02C0EEFF03C0EEFF4B
:101BE00034C4E9FF35C4EAFF040EEF6E0101000EB4
:101BF000D880D555000ED6551DE234C4E9FF35C452
:101C0000EAFF250EE926000EEA22EF8634C4E9FF3A
:101C100035C4EAFF120ED5C1EBFF130ED6C1EBFFA0
:101C200034C4E9FF35C4EAFF250EE926000EEA2296
:101C3000EF8402D090EC24F002D090EC24F05BD240
:101C400034C4E9FF35C4EAFFEF50006E016A00BEFC
:101C50000168030E001801E1015001E087D0D3C1F3
:101C6000E9FFD4C1EAFF0D0EE926000EEA22EF508B
:101C7000020B01E0010E006E016A0050011073E0DA
:101C8000242B000E25232623272334C4E9FF35C443
:101C9000EAFF180EE926000EEA2224C4EEFF25C44E
:101CA000EEFF26C4EEFF27C4EEFFD3C1E9FFD4C187
:101CB000EAFF0D0EE926000EEA22EF50100B01E0BC
:101CC000010E006E016A0050011009E0100E366F1F
:101CD00034C4E9FF35C4EAFF040EEF6E1DD0120EC6
:101CE000366F34C4E9FF35C4EAFF020EEF6E282BCD
:101CF000000E29232A232B2334C4E9FF35C4EAFF2D
:101D0000140EE926000EEA2228C4EEFF29C4EEFFD5
:101D10002AC4EEFF2BC4EEFF0101000ED880D5557A
:101D2000000ED6551DE234C4E9FF35C4EAFF250E86
:101D3000E926000EEA22EF8634C4E9FF35C4EAFF43
:101D4000120ED5C1EBFF130ED6C1EBFF34C4E9FF71
:101D500035C4EAFF250EE926000EEA22EF8402D000
:101D600090EC24F002D090EC24F0C5D1D3C1E9FF6F
:101D7000D4C1EAFF040EE926000EEA22EECF00F0FD
:101D8000EECF01F0EECF02F0EFCF03F034C4E9FF65
:101D900035C4EAFF180EE926000EEA220050EE18BC
:101DA00009E10150EE1806E10250EE1803E103507C
:101DB000EE1800E103E090EC24F0E3D134C4E9FF35
:101DC00035C4EAFF180EE926000EEA2224C4EEFF0D
:101DD00025C4EEFF26C4EEFF27C4EEFF34C4E9FF9E
:101DE00035C4EAFFEF50006E016A00BE0168040EC0
:101DF000001801E1015001E0DAD0D3C1E9FFD4C1FC
:101E0000EAFF0D0EE926000EEA22EF50100B01E06A
:101E1000010E006E016A0050011029E034C4E9FF90
:101E200035C4EAFF0F0EEB50006E016AFF0E00187A
:101E300001E101501CE034C4E9FF35C4EAFF0F0E94
:101E4000EB500101E66F7FEC24F034C4E9FF35C4A8
:101E5000EAFF0F0EE926000EEA22EF6834C4E9FF1C
:101E600035C4EAFF250EE926000EEA22EF82D3C12F
:101E7000E9FFD4C1EAFF0D0EE926000EEA22EF5079
:101E8000010B006E016A0050011031E00401110ED7
:101E9000366F34C4E9FF35C4EAFF140EE926000E9C
:101EA000EA22EFCF28F4EE2AEFCF29F4EE22EFCF8B
:101EB0002AF4EE22EFCF2BF4EF2234C4E9FF35C42D
:101EC000EAFF180EE926000EEA22EF2AEECF24F4EC
:101ED000EF22EECF25F4EF22EECF26F4EF22EFCF64
:101EE00027F434C4E9FF35C4EAFF0A0EEF6E01019E
:101EF000000ED880D555000ED65556E234C4E9FF01
:101F000035C4EAFF250EE926000EEA22EF50080B41
:101F100001E0010E006E016A0050011020E134C49E
:101F2000E9FF35C4EAFF250EE926000EEA22EF8616
:101F300034C4E9FF35C4EAFF120ED5C1EBFF130E1E
:101F4000D6C1EBFF34C4E9FF35C4EAFF250EE9260C
:101F5000000EEA22EF840401100E366F24D0040133
:101F6000366B34C4E9FF35C4EAFF140EE926000ECF
:101F7000EA2230C4EEFF31C4EEFF32C4EEFF33C4B8
:101F8000EEFF34C4E9FF35C4EAFF180EE926000E5F
:101F9000EA222CC4EEFF2DC4EEFF2EC4EEFF2FC4A8
:101FA000EEFF90EC24F002D090EC24F0A4D034C4E6
:101FB000E9FF35C4EAFFEF50006E016A00BE016818
:101FC0000A0E001801E101501AE190EC24F0D3C18F
:101FD000E9FFD4C1EAFF0D0EE926000EEA22EF5018
:101FE000100B01E0010E006E016A0050011006E0C6
:101FF00034C4CEF135C4CFF18FEC0BF07CD034C4B7
:10200000E9FF35C4EAFFEF50006E016A00BE0168C7
:10201000050E001801E1015047E190EC24F0D3C116
:10202000E9FFD4C1EAFF0D0EE926000EEA22EF50C7
:10203000010B006E016A0050011035E00401100E22
:10204000366F34C4E9FF35C4EAFF180EE926000EE6
:10205000EA22EF2AEECF24F4EF22EECF25F4EF228E
:10206000EECF26F4EF22EFCF27F4D3C1E9FFD4C19E
:10207000EAFF0D0EE926000EEA22EF50100B01E0F8
:10208000010E006E016A0050011007E034C4CEF169
:1020900035C4CFF18FEC0BF006D034C4E9FF35C462
:1020A000EAFF060EEF6E27D034C4E9FF35C4EAFF1D
:1020B000EF50006E016A00BE0168060E001801E1D3
:1020C000015019E190EC24F0D3C1E9FFD4C1EAFF3B
:1020D0000D0EE926000EEA22EF50100B01E0010E72
:1020E000006E016A0050011006E034C4CEF135C420
:1020F000CFF18FEC0BF002D090EC24F004013651BC
:10210000006E016A0150000AE8AE02D0013405D029
:10211000000ED8800054000E015433E20101C46B5C
:10212000C56B0101C369040136510101C26F24C4AA
:10213000BEF125C4BFF126C4C0F127C4C1F128C433
:10214000BAF129C4BBF12AC4BCF12BC4BDF1D3C17F
:10215000E9FFD4C1EAFFEECFB8F1EDCFB9F1D3C1B9
:10216000E9FFD4C1EAFF020EE926000EEA22EECF13
:10217000B6F1EDCFB7F1D1C1B4F1D2C1B5F1DEEC1A
:0421800007F0120052
:0C2184000401036B0351006E016A01505E
:10219000000AE8AE02D0D89004D0020E005C000E17
:1021A000015826E2500E01019E6F9F6BF0EC00F08B
:1021B000E66E040103510A0DF3CFE9FFF4CFEAFF05
:1021C000400EE926020EEA22E552E750EF6E035177
:1021D0000A0DF3CFE9FFF4CFEAFF400EE926020E25
:1021E000EA22030EE926000EEA22EF6A032BCCD77F
:1021F00012000401B36BB351006E016A0150000A72
:10220000E8AE02D0D89004D0020E005C000E015857
:1022100007E2B3510201546F04D80401B32BEBD78A
:102220001200020154510A0DF3CF61F4F4CF62F4AD
:10223000400E04016127020E6223010E546F54C444
:1022400000F0016A00BE01680050011001E18FD268
:102250000401546B61C4E9FF62C4EAFFEF5001015D
:10226000A06F66EC01F000090AE161C4E9FF62C4F5
:10227000EAFF030EE926000EEA22EF6A78D261C473
:10228000E9FF62C4EAFF030EEB50006E016A00BE74
:102290000168090E001801E1015001E13DD2010E73
:1022A000001801E1015001E10FD20B0E001801E10D
:1022B000015001E155D1020E001801E1015001E188
:1022C000FED0005001E1015001E050D261C4E9FFAD
:1022D00062C4EAFFEF500101AF6F84EC04F0000923
:1022E00001E1ECD00401010E546F526B536B0401F9
:1022F000500E525D000E535917E252C4ADF153C453
:10230000AEF1522B000E5323000E0101AD27040E37
:10231000AE2361C4E9FF62C4EAFFEF500101AC6F74
:102320001AEC04F0000902E1000E01D0010E006E6B
:10233000016A0050011001E0DAD7000E04015225B5
:10234000E96E040E5321EA6EEF6A61C4E9FF62C4CC
:10235000EAFFEF500101A66F93EC03F061C4E9FFBF
:1023600062C4EAFF030EE926000EEA22020EEF6EB7
:102370000401050E5F6F61C4E9FF62C4EAFF090E44
:10238000E926000EEA22E9CF5DF2EACF5EF2020111
:102390005F0E5B6F040E5C6F0201550E596F040EE9
:1023A0005A6F0201000E576F040E586F2BDB0401A9
:1023B000516F51C400F0016A00BE01680050011065
:1023C00001E07CD05F51006E016A0150000AE8AE66
:1023D00002D0013405D0010ED8800054000E015403
:1023E00014E25F510001B56F0001550EB36F040E8A
:1023F000B46F3DEC19F061C4E9FF62C4EAFF090E55
:10240000E926000EEA22030EEF6E55C4B9F256C457
:10241000BAF2D2EC35F0F3CF00F0F4CF01F061C4A2
:10242000E9FF62C4EAFF010E00C0EBFF020E01C02B
:10243000EBFF61C4E9FF62C4EAFFEE52FF0EEE1843
:1024400002E1FF0EED1814E161C4E9FF62C4EAFF86
:10245000080EE926000EEA22EF6A61C4E9FF62C4B1
:10246000EAFF030EE926000EEA22020EEF6E26D0E6
:1024700061C4E9FF62C4EAFFEE52EE50ED1014E1D0
:1024800061C4E9FF62C4EAFF080EE926000EEA22F1
:10249000030EEF6E61C4E9FF62C4EAFFE926000E95
:1024A000EA22020EEF6E0AD061C4E9FF62C4EAFFBD
:1024B000030EE926000EEA220B0EEF6E57D161C41F
:1024C000E9FF62C4EAFFEF500101A36FDFEC02F005
:1024D000000945E061C4E9FF62C4EAFF080EEB5061
:1024E000E96EEA6AD890E936EA36D20EE926020E9B
:1024F000EA22EECF63F4EDCF64F4040163C4F6FF87
:1025000064C4F7FF632B000E64230800F5CF00F0CE
:10251000016A00BE016800C060F400500DE0605127
:102520000101A56F61C4E9FF62C4EAFFEF50010138
:10253000A46F0EEC03F0E1D761C4E9FF62C4EAFFC7
:10254000EF500101A26F08EC02F061C4E9FF62C420
:10255000EAFF030EE926000EEA22090EEF6E06D10D
:1025600061C4E9FF62C4EAFFEF500101A36FDFEC31
:1025700002F0000901E1A7D00401010E546F606B65
:102580006051006E016A1F0E005C000E015816E2D9
:102590006051F76A960FF66E790EF7220800F55033
:1025A0000101A56F61C4E9FF62C4EAFFEF500101B8
:1025B000A46F0EEC03F00401602BE2D761C4E9FFC5
:1025C00062C4EAFF090EEB50140DF3CFF6FFF4CF0F
:1025D000F7FF0A0EF626790EF722F6CF63F4F7CF4F
:1025E00064F4040163C4F6FF64C4F7FF632B000EB8
:1025F00064230800F5CF00F0016A00BE016800C046
:1026000060F400500DE060510101A56F61C4E9FF65
:1026100062C4EAFFEF500101A46F0EEC03F0E1D7B2
:10262000606B6051006E016A040E005C000E015880
:1026300016E26051F76AB60FF66E790EF7220800BF
:10264000F5500101A56F61C4E9FF62C4EAFFEF50D4
:102650000101A46F0EEC03F00401602BE2D761C40A
:10266000E9FF62C4EAFF090EEB50006E016A030E37
:10267000001801E101500BE161C4E9FF62C4EAFF07
:10268000070EE926000EEA22010EEF6E09D061C4A2
:10269000E9FF62C4EAFF070EE926000EEA22EF6AAC
:1026A00061C4E9FF62C4EAFF040EE926000EEA22D3
:1026B000030EEF6E61C4E9FF62C4EAFFE926000E73
:1026C000EA22010EEF6E52D061C4E9FF62C4EAFF54
:1026D000EF500101AF6F84EC04F0000909E061C420
:1026E000E9FF62C4EAFFEF500101A66F93EC03F02B
:1026F00061C455F262C456F23BD800090CE083EC89
:1027000036F061C4E9FF62C4EAFF030EE926000E59
:10271000EA22090EEF6E2AD061C4E9FF62C4EAFF23
:10272000EF500101A06F66EC01F000091EE061C4EA
:10273000E9FF62C4EAFFEF500101A36FDFEC02F092
:10274000000913E061C4E9FF62C4EAFFEF50010130
:10275000A16F83EC01F061C4E9FF62C4EAFF030EDC
:10276000E926000EEA220A0EEF6E00D068D51200AC
:1027700055C2E9FF56C2EAFFEE52EECFB4F2EDCFFA
:10278000B5F255C2E9FF56C2EAFFEF500101A36F4F
:10279000DFEC02F0000901E128D10401B16B55C260
:1027A000E9FF56C2EAFF040EEB50006E016A080E04
:1027B000001801E1015014E08EEC36F00401B26F14
:1027C0000201B41D01E1B51D0BE155C2E9FF56C27E
:1027D000EAFFEF500101A26F08EC02F0010E11D1E7
:1027E00055C2E9FF56C2EAFF070EEB50006E016AC0
:1027F0000050011001E1EBD055C2E9FF56C2EAFFDB
:10280000040EEB50006E016A080E001801E1015041
:1028100001E181D0060E001801E1015057E0050EDC
:10282000001801E101501DE0030E001801E1015004
:1028300001E0B6D00401B251006E016A250E001805
:1028400001E101500BE155C2E9FF56C2EAFF040E57
:10285000E926000EEA22050EEF6E02D0010EB16FDE
:10286000A0D00401B251006E016A250E001801E1EA
:1028700001500DE1010EB16F55C2E9FF56C2EAFFEA
:10288000040EE926000EEA22030EEF6E1ED0B251AE
:10289000006E016A300E005E000E015A040ED890E0
:1028A00000360136E804FBE155C2E9FF56C2EAFFF3
:1028B000080E00C0EBFF55C2E9FF56C2EAFF040E46
:1028C000E926000EEA22060EEF6E6BD00401B2512B
:1028D000006E016A300E005E000E015A55C2E9FF1B
:1028E00056C2EAFF080EE926000EEA220050EF1257
:1028F00055C2E9FF56C2EAFF040EE926000EEA229D
:10290000080EEF6E55C2E9FF56C2EAFF050EEB6AEC
:10291000060EEB6A46D00001B20EB96F040EBA6F14
:1029200055C2E9FF56C2EAFF050EE926000EEA226B
:10293000EECFB7F0EDCFB8F055C2E9FF56C2EAFFCF
:10294000080EEB500001B66FBDEC19F0F3CF00F0AC
:10295000F4CF01F055C2E9FF56C2EAFF050E00C0F0
:10296000EBFF060E01C0EBFF0401010EB16F55C273
:10297000E9FF56C2EAFF050EE926000EEA22FF0E25
:10298000EE1802E1FF0EED180AE155C2E9FF56C24A
:10299000EAFF040EE926000EEA22030EEF6E01D0D4
:1029A000FFD7B1C400F0016A00BE016800500110F9
:1029B0000DE00401B2510101A56F55C2E9FF56C2F5
:1029C000EAFFEF500101A46F0EEC03F00DD00401FB
:1029D000B2510101A56F55C2E9FF56C2EAFFEF509F
:1029E0000101A46F0EEC03F0CCD655C2E9FF56C22C
:1029F000EAFF010EB4C2EBFF020EB5C2EBFF000E00
:102A000000D012000401666B686B696B656B030E86
:102A1000E66EE66ABB0E006E790E016E026A00C0B9
:102A2000E6FF01C0E6FF02C0E6FF57C2E6FF58C25C
:102A3000E6FF09EC3BF0F56E070EE15EF55000098C
:102A400008E1040E02015727000E58230401676BAA
:102A500002D0020EF1D157C2E9FF58C2EAFFEF508F
:102A6000006E016A200E001801E1015005E102012B
:102A7000572B000E5823EFD757C2E9FF58C2EAFF81
:102A8000EF5004016A6F6A51066E076A200E06183D
:102A900001E1075006E06A51086E096A0850091002
:102AA00002E1000E01D0010E046E056A045005100B
:102AB00008E06A510A6E0B6A0D0E0A1801E10B500C
:102AC00002E1000E01D0010E026E036A02500310F3
:102AD00008E06A510C6E0D6A0A0E0C1801E10D50E7
:102AE00002E1000E01D0010E006E016A00500110DB
:102AF00001E10CD16551006E016A5BC2E9FF5CC265
:102B0000EAFFEF50000101AF02D0D89003D0005D82
:102B1000000E015901E3FAD004016651006E016A0A
:102B2000020E001801E101504AE0010E001801E117
:102B3000015034E0005001E1015001E0DBD065516B
:102B4000020D02015951F324E96E5A51F420EA6E44
:102B500057C2EEFF58C2EDFF57C2E9FF58C2EAFF65
:102B6000EF5004016A6F6A51026E036A2F0E021859
:102B700001E103500AE06A51046E056A5C0E041814
:102B800001E1055002E0000E01D0010E006E016A65
:102B90000050011002E0010E666FACD06551652B4C
:102BA000020D02015951F324E96E5A51F420EA6EE4
:102BB00057C2EEFF58C2EDFF0401020E666F57C206
:102BC000E9FF58C2EAFFEF506A6F6A51026E036A6A
:102BD0003F0E021801E103500AE06A51046E056AD3
:102BE000260E041801E1055002E0000E01D0010E8E
:102BF000006E016A0050011008E057C2E9FF58C298
:102C0000EAFFEF6A010E666F74D06A51006E016AC6
:102C10002B0E001801E1015007E1200E57C2E9FF19
:102C200058C2EAFFEF6E65D06A51026E036A2E0E3B
:102C3000021801E1035008E16551046E056A010EB6
:102C4000041801E1055002E0000E01D0010E006EF3
:102C5000016A0050011009E00201572B000E5823B1
:102C600057C268F458C269F444D06A51006E016AD0
:102C70003D0E001801E1015008E157C2E9FF58C2BA
:102C8000EAFFEF6A010E666F34D06A51026E036A82
:102C90002F0E021801E103500AE06A51046E056A22
:102CA0005C0E041801E1055002E0000E01D0010E97
:102CB000006E016A005001101CE0010E0201036A5F
:102CC0005725026E5851032204016551006E016AB6
:102CD0000006000E015AD890003601360201595103
:102CE0000024E96E5A510120EA6E02C0EEFF03C0D3
:102CF000EDFF00D00201572B000E582357C2E9FF09
:102D000058C2EAFFEF5004016A6FBDD657C2E9FF0F
:102D100058C2EAFFEF6A070E5DC2E9FF5EC2EAFF32
:102D2000EF6E04016851691143E068C4E6FF69C4AD
:102D3000E6FFAFEC3BF0E552E552F3CF68F4F4CF99
:102D400069F40401EE0E6B6F780E6C6F6A6B6A515A
:102D5000006E016A070E005C000E015829E2030EA6
:102D6000E66EE66A6BC400F06CC401F0026A00C053
:102D7000E6FF01C0E6FF02C0E6FF68C4E6FF69C4E3
:102D8000E6FF09EC3BF0F56E070EE15EF550000939
:102D900008E104016A515DC2E9FF5EC2EAFFEF6E1D
:102DA00007D0040E04016B27000E6C236A2BCFD7CB
:102DB0006551006E016A0050011031E1090EE66EA6
:102DC000E66ABF0E006E790E016E026A00C0E6FF71
:102DD00001C0E6FF02C0E6FF59C2E9FF5AC2EAFF9E
:102DE000EECFE6FFEFCFE6FF53EC3BF0F56E070EBC
:102DF000E15EF55059C2E9FF5AC2EAFFEE50EFCF4B
:102E0000EAFFE96E090EE926000EEA22EF6A010EDA
:102E10005DC2E9FF5EC2EAFFEF6E0401652B6551FA
:102E20005BC2E9FF5CC2EAFFEF6E67C400F0016AB3
:0A2E300000BE0168005000D012003F
:062E3A00DACFE4FFE2CF55
:102E4000DAFFE9CFE4FFEACFE4FF00EE00F0160E70
:102E5000E80403E3EECFE4FFFBD7E6528BEC3DF052
:102E6000E55200EE15F0160EE80403E3E5CFEDFFA2
:102E7000FBD7E5CFEAFFE5CFE9FFE5CFDAFF1100A9
:102E8000AC50020B01E0010E006E016A005001100F
:102E900001E1F6D700019D51AD6E120000019EC008
:102EA000E9FF9FC0EAFF9E2B000E9F23EF50040115
:102EB000226F000905E0225100019D6FE1DFEED78E
:102EC000120034DB71EC3DF0CCEC35F04FDB81507F
:102ED000200B01E0010E006E016A005001100EE1AE
:102EE0000201C00EDA6F4FEC39F00201370EDD6FD0
:102EF000740EDE6FBCEC39F008EC1DF029EC33F0F9
:102F0000C2EC10F000019851010B006E016A0050F4
:102F100001100DE00201C00EDA6F4FEC39F0020132
:102F2000260EDD6F740EDE6FBCEC39F006D00201A8
:102F3000010E8E6F0101070EFB6F7AEC3DF002016E
:102F40008F511A5C006E90511B58016E91511C58A4
:102F5000026E92511D58036E320E005C000E015835
:102F6000000E0258000E03580BE37AEC3DF01AC035
:102F70008FF21BC090F21CC091F21DC092F28978B2
:102F800034EC33F0F9EC10F023D90101FE51006E5E
:102F9000016A02018E51026E036A0250001802E1BA
:102FA0000350011836E00001010EA26F0001800EEF
:102FB000A06F000EA16F2FD80101FE5102018E6F8C
:102FC00000019851010B006E016A0050011021E0D0
:102FD0000201CE0EDA6F4FEC39F002018E51006E15
:102FE000016A0150000AE8AE02D0D89004D00A0E5F
:102FF000005C000E015807E2300E8E250201DF6FE3
:10300000D8EC39F006D0410E8E250201DF6FD8ECE6
:1030100039F093D71200A2C000F0016A00BE016827
:10302000005001100CE00201C00EDA6F4FEC39F0D5
:103030000201460EDD6F740EDE6FBCEC39F002014A
:10304000C00EDA6F4FEC39F01A0EE66E040EE66E23
:10305000A0C0E9FFA1C0EAFFEF50E66EE66A65ECAA
:1030600037F0E552E552E552E552A2C000F0016AA0
:1030700000BE0168005001100DE002011A0EDB6F66
:10308000040EDC6FA1EC39F002012E0EDF6FD8ECDC
:1030900039F00AD000011A0E9E6F040E9F6FFEDEFB
:1030A00000012E0E9D6FECDE1A0EE66E040EE66E2B
:1030B000A0C0E9FFA1C0EAFF010EE926000EEA2246
:1030C000EF50E66EE66A65EC37F0E552E552E55200
:1030D000E552A2C000F0016A00BE01680050011074
:1030E0000DE002011A0EDB6F040EDC6FA1EC39F06B
:1030F00002012E0EDF6FD8EC39F00AD000011A0E53
:103100009E6F040E9F6FCADE00012E0E9D6FB8DE0B
:103110001A0EE66E040EE66EA0C0E9FFA1C0EAFF3B
:10312000020EE926000EEA22EF50E66EE66A65EC32
:1031300037F0E552E552E552E552A2C000F0016ACF
:1031400000BE0168005001100DE002011A0EDB6F95
:10315000040EDC6FA1EC39F002012E0EDF6FD8EC0B
:1031600039F00AD000011A0E9E6F040E9F6F96DE92
:1031700000012E0E9D6F84DE1A0EE66E040EE66EC2
:10318000A0C0E9FFA1C0EAFF030EE926000EEA2273
:10319000EF50E66EE66A65EC37F0E552E552E5522F
:1031A000E552A2C000F0016A00BE016800500110A3
:1031B00008E002011A0EDB6F040EDC6FA1EC39F09F
:1031C00006D000011A0E9E6F040E9F6F67DE12007C
:1031D000810EC26E0401640E006F005100070009E9
:1031E00001E0FBD7C284C250040B01E0010E006E67
:1031F000016A0050011001E0F6D7C3500401006FCE
:10320000C450016FA30EE66E000EE66E00C4E6FF2A
:1032100001C4E6FF65EC37F0E552E552E552E552B0
:10322000840EC16E890EC26E0401640E006F0051DF
:103230000007000901E0FBD7C284C250040B01E083
:10324000010E006E016A0050011001E0F6D7C35074
:103250000401006FC450016FAB0EE66E000EE66E07
:1032600000C4E6FF01C4E6FF65EC37F0E552E55225
:10327000E552E5528E0EC16E1200B3C0E9FFB4C034
:10328000EAFFEE50EFCFEAFFE96EEF50006E016A01
:10329000300E005E000E015A00C065F40401655155
:1032A000006E016A010E001801E1015064E0005057
:1032B00001E101501DE00A0EE66EE66A640E006E42
:1032C000740E016E026A00C0E6FF01C0E6FF02C094
:1032D000E6FFB3C0E9FFB4C0EAFFEECFE6FFEFCFF1
:1032E000E6FF53EC3BF0F56E070EE15EF55044D07F
:1032F000020E0001EA6AB325E96EB451EA22EE50EB
:10330000EFCFEAFFE96EEF50006E016A300E005E0B
:10331000000E015A00C066F404016651006E016A95
:10332000010E001801E1015007E0005001E10150D9
:1033300001E004D0897602D0897400D00D0EE66ECB
:10334000E66A570E006E740E016E026A00C0E6FF58
:1033500001C0E6FF02C0E6FFB3C0E9FFB4C0EAFF68
:10336000EECFE6FFEFCFE6FF53EC3BF0F56E070E36
:10337000E15EF55001D000D012000001B651006EA0
:10338000016A040E001801E1015001E1B0D0030E02
:10339000001801E1015074E0020E001801E1015033
:1033A00038E0010E001801E101501CE0005001E17D
:1033B000015001E0B3D08950080B01E0010E006E0E
:1033C000016A0050011007E0300EB9C0E9FFBAC031
:1033D000EAFFEF6E06D0310EB9C0E9FFBAC0EAFFCE
:1033E000EF6E9CD08950040B01E0010E006E016A63
:1033F0000050011007E0300EB9C0E9FFBAC0EAFF83
:10340000EF6E06D0310EB9C0E9FFBAC0EAFFEF6E29
:1034100085D0B751B81102E1B76BB86BB751EA6A02
:10342000A30FE96E000EEA22EFCF00F0016A00BEA2
:1034300001680050B9C0E9FFBAC0EAFFEF6EB751AA
:10344000EA6AA30FE96E000EEA22EFCF00F0016AEC
:1034500000BE01680050011007E10068016800C06B
:10346000F3FF01C0F4FF61D0B7C000F0B8C001F0B5
:10347000B72B000EB823B7C0F3FFB8C0F4FF55D088
:10348000B751B81102E1B76BB86BB751EA6AAB0F2D
:10349000E96E000EEA22EFCF00F0016A00BE01687B
:1034A0000050B9C0E9FFBAC0EAFFEF6EB751EA6A4F
:1034B000AB0FE96E000EEA22EFCF00F0016A00BE0A
:1034C00001680050011007E10068016800C0F3FFC7
:1034D00001C0F4FF2AD0B7C000F0B8C001F0B72B8C
:1034E000000EB823B7C0F3FFB8C0F4FF1ED0815060
:1034F000200B01E0010E006E016A0050011007E090
:10350000310EB9C0E9FFBAC0EAFFEF6E06D0300E47
:10351000B9C0E9FFBAC0EAFFEF6E00D000680168E9
:1035200000C0F3FF01C0F4FF00D012008E0EC16E88
:10353000030E926E809A89848986F19E09EC39F097
:103540000201800EDA6F4FEC39F00201160EDD6FCA
:10355000740EDE6FBCEC39F0200EAC6E900EAB6ECC
:103560000F0EAF6ED56AF28EF28C120000010A0EB9
:10357000806F816F050E826F0F0E836F8A698B6972
:103580008C698D6B0A0E8E6F8F6F050E906F0F0E0C
:10359000916F846B040E856FA30E866F876B886BAB
:1035A000896B988112000001BBC0F6FFBCC0F7FF19
:1035B000BB2B000EBC230800F5CF00F0016A00BE53
:1035C000016800C01AF4005006E004011A5100011D
:1035D0009D6F56DCE8D7120004011B6B9E50200B38
:1035E00001E0010E006E016A0050011001E1F6D702
:1035F000AE5004011A6F1A51026E036A0D0E0218C2
:1036000001E103500AE01A51046E056A0A0E04181B
:1036100001E1055002E0000E01D0010E006E016ACA
:103620000050011001E01CD01B2B1A51E66E000166
:10363000BDC0E9FFBEC0EAFFBD2B000EBE23E552B0
:10364000E750EF6EBDC0E9FFBEC0EAFFEF6ABF51B1
:10365000BF07006E016A0050011001E101D0BED722
:1036600004011B5100D01200C0C01BF4C1C01CF4E7
:1036700004011D6BC0C0E9FFC1C0EAFFEFCF00F03D
:10368000016A00BE016800C01AF4005061E0040144
:103690001A51006E016A2E0E001801E101502CE152
:1036A0000001C0C0E9FFC1C0EAFFC02B000EC1236A
:1036B000EF6A1BC4E6FF1CC4E6FFF0EC36F0E552EF
:1036C000E552F350E66EC2C0E9FFC3C0EAFFE9CF9E
:1036D00000F0EACF01F004011D511D2B0F01002461
:1036E000E96F000E0120EA6FE552E750EF6EC0C0AF
:1036F0001BF4C1C01CF427D01A51026E036A035098
:10370000000AE8AE02D0D89004D0300E025C000E61
:10371000035811E31A51046E056A0550000AE8AE19
:1037200002D0053405D0390ED8800454000E05545B
:1037300002E3000E01D0010E006E016A005001107C
:1037400002E0000E32D00001C02B000EC12392D740
:103750001BC4E6FF1CC4E6FFF0EC36F0E552E55270
:10376000F350E66EC2C0E9FFC3C0EAFFE9CF00F044
:10377000EACF01F004011D510F010024E96F000E92
:103780000120EA6FE552E750EF6E04011D51026E11
:10379000036A030E021801E1035002E0000E01D09B
:1037A000010E006E016A005000D012009E50200BE6
:1037B00001E0010E006E016A0050011001E1F6D730
:1037C000AE500401006F0051026E036A0350000AFC
:1037D000E8AE02D0D89004D0310E025C000E03583F
:1037E0000EE30051046E056A0550000AE8AE02D0EF
:1037F000D89004D0390E045C000E055802E3000E88
:1038000001D0010E006E016A0050011003E000516A
:1038100003D002D0390E00D0120000010D0E9D6FB2
:1038200040EC17F000010A0E9D6F40EC17F0C4C089
:10383000E9FFEA6AE9BEEA68300EE95E000EEA5A7C
:10384000E906EA5AD890E936EA36930EE926020EDE
:10385000EA22EECFBBF0EDCFBCF0A5DEC4C000F095
:10386000016A00BE0168380E001801E1015001E153
:10387000CDD0370E001801E1015001E1C6D0360E5F
:10388000001801E1015001E1BDD0350E001801E141
:10389000015001E1B4D0340E001801E101505EE0A6
:1038A000330E001801E1015053E0320E001801E11F
:1038B000015048E0310E001801E1015001E0A7D0AD
:1038C000000EE66E040EE66E92C0E6FF93C0E6FFC1
:1038D00065EC37F0E552E552E552E5520001000E85
:1038E0009E6F040E9F6F4EEC17F00001290E9D6F26
:1038F00040EC17F000013A0E9D6F40EC17F000010C
:10390000200E9D6F40EC17F00001140EBF6F0001F8
:10391000000EBD6F040EBE6F5FDE000912E0000EE8
:10392000E66E040EE66EF0EC36F0E552E552F3CFAB
:1039300092F0F4CF93F000019351886F9251896F08
:1039400066D03ED00401800E186F000E196F0BD0A8
:1039500004018E0E186F000E196F05D004018A0E37
:10396000186F000E196F0001A26B18C4A0F019C4E3
:10397000A1F00BEC18F00001290E9D6F40EC17F040
:1039800000013A0E9D6F40EC17F00001200E9D6F74
:1039900040EC17F00001140EBF6F0001000EBD6F68
:1039A000040EBE6F19DE0001140EC26F040EC36F49
:1039B0000001000EC06F040EC16F56DE000912E157
:1039C0000001C70EBB6F750EBC6FEDDD9E50200B66
:1039D00001E0010E006E016A0050011001E1F6D70E
:1039E000AE500CD018C4E9FF19C4EAFF14C4EEFFAE
:1039F00015C4EEFF16C4EEFF17C4EEFF08D0000199
:103A0000988105D00001989102D001D000D0120019
:103A100000016E0EBB6F740EBC6FC5DDC7DE040106
:103A2000236F23C400F0016A00BE0168390E00183C
:103A300001E1015008E023C400F0016A00BE016802
:103A400000C0C4F0EADE23C400F0016A00BE0168D1
:103A5000380E001801E10150DBE112004B0EE66E5A
:103A60009FEC3DF0E5521200140EE66E9FEC3DF027
:103A7000E5521200F29E050EE66EBDEC3DF0E552F9
:043A8000F28E1200B0
:0C3A8400FBC100F0016A00BE0168070EE3
:103A9000001801E1015001E112D00101FC51006E5A
:103AA000016AFF0E001801E1015005E0FC5102011E
:103AB000336F25EC28F00101FC69FB6BFE6B1200F3
:103AC000FBC100F0016A00BE0168060E001801E1AA
:103AD000015001E15FD1050E001801E1015001E143
:103AE000D4D0040E001801E1015001E1B4D0030E5E
:103AF000001801E1015001E17DD0020E001801E142
:103B0000015054E0010E001801E1015033E0005073
:103B100001E1015001E06CD1040100690169026911
:103B20000369046905690669076908690969020189
:103B3000676B686B696B6A6B430E0201316F326BA6
:103B40000201000E2F6F040E306F440E02012D6F24
:103B50002E6BADEC27F00101FC6F7AEC3DF01AC042
:103B600073F21BC074F21CC075F21DC076F2010125
:103B7000010EFB6F7AEC3DF0020173511A5C006E8E
:103B800074511B58016E75511C58026E76511D58A8
:103B9000036E140E005C000E0158000E0258000E59
:103BA000035803E30101020EFB6F22D102016751AA
:103BB000681169116A1104E00101040EFB6F19D04C
:103BC0000101FC5102012C6F84EC23F0000911E08B
:103BD0000201010E776F3CDB7AEC3DF01AC073F204
:103BE0001BC074F21CC075F21DC076F20101030EF9
:103BF000FB6FFED07AEC3DF0020173511A5C006E4F
:103C000074511B58016E75511C58026E76511D5827
:103C1000036EC80E005C000E0158000E0258000E24
:103C2000035803E30101020EFB6F0101FC51020185
:103C3000356F42EC29F000090DE0E3D8006E016A0F
:103C4000020E001801E1015004E10101040EFB6FB6
:103C500002D0CED0CDD00101FC5102012C6F84ECFA
:103C600023F0000911E00201030E776FF1DA7AEC1C
:103C70003DF01AC073F21BC074F21CC075F21DC077
:103C800076F20101050EFB6FB3D00101FC51020178
:103C9000356F42EC29F0000961E0B3D804010A6FE6
:103CA0000A51006E016A060E001801E1015004E19C
:103CB0000101040EFB6F51D00A51006E016A050E1E
:103CC000001801E1015049E10101FC510201336F8B
:103CD00025EC28F00101FC697AEC3DF01AC073F282
:103CE0001BC074F21CC075F21DC076F20101060EF5
:103CF000FB6F020167510001806F020168510001F2
:103D0000816F020169510001826F02016A51000155
:103D1000836F02016F5100018A6F0201705100012F
:103D20008B6F0201715100018C6F02017251000111
:103D30008D6F02016B5100018E6F02016C51000109
:103D40008F6F02016D510001906F02016E510001F1
:103D5000916F0101FD81FE2B4BD01BD07AEC3DF021
:103D6000020173511A5C006E74511B58016E75513B
:103D70001C58026E76511D58036EC80E005C000E72
:103D80000158000E0258000E035803E30101020E11
:103D9000FB6F2ED07AEC3DF0020173511A5C006E7D
:103DA00074511B58016E75511C58026E76511D5886
:103DB000036E640E005C000E0158000E0258000EE7
:103DC000035816E36307000E645B655B665B635133
:103DD00064116511661102E10101FB6B7AEC3DF0A3
:103DE0001AC073F21BC074F21CC075F21DC076F2CB
:103DF00012000101080EFB6FFC510201336F25EF29
:103E000028F004010D6B02013C0E636F646B656B5F
:103E1000666B02010B0E366F040E376F5EEC29F0F5
:103E200004010B51006E016A020E001801E10150FD
:103E300001E0E0D10C6B0C51006E016A0150000AE8
:103E4000E8AE02D0D89004D00F0E005C000E0158EE
:103E50000AE202010B0E366F040E376F5EEC29F09A
:103E600004010C2BE8D70201670E366F020E376F84
:103E70005EEC29F00201680E366F020E376F5EECC1
:103E800029F00201690E366F020E376F5EEC29F0E1
:103E900002016A0E366F020E376F5EEC29F00401E4
:103EA0000C6B0C51006E016A0150000AE8AE02D0A2
:103EB000D89004D0080E005C000E01580AE20201FE
:103EC0000B0E366F040E376F5EEC29F004010C2BDD
:103ED000E8D70C6B0C51006E016A0150000AE8AE85
:103EE00002D0D89004D0060E005C000E01581DE2EE
:103EF00002010B0E366F040E376F5EEC29F00401E1
:103F00000B51006E016A0C51EA6A840FE96E000ED3
:103F1000EA22EF50026E036A0250001802E10350D9
:103F2000011801E090D10C2BD5D70C6B0C51006E11
:103F3000016A0150000AE8AE02D0D89004D0CE0E3B
:103F4000005C000E01580AE202010B0E366F040EEF
:103F5000376F5EEC29F004010C2BE8D70E6B0201E1
:103F60000B0E366F040E376F5EEC29F004010B5117
:103F7000006E016A330E001801E1015001E1DCD04E
:103F8000E868001801E1015001E1D3D0360E0018B5
:103F900001E1015001E19ED0030E001801E1015042
:103FA00054E0010E001801E1015020E0350E001828
:103FB00001E1015001E001D102010B0E366F040E48
:103FC000376F5EEC29F004010B51006E016A010E9F
:103FD000001801E1015008E102010D0E366F040ED8
:103FE000376F5EEC29F001D02ED1FBD002010B0E11
:103FF000366F040E376F5EEC29F004010B51006E32
:10400000016A040E001801E101501DE102016F0E6A
:10401000366F020E376F5EEC29F00201700E366FBC
:10402000020E376F5EEC29F00201710E366F020E40
:10403000376F5EEC29F00201720E366F020E376F99
:104040005EEC29F001D0FFD0CCD002010B0E366F10
:10405000040E376F5EEC29F004010B51006E016A0B
:104060000150000AE8AE02D0D89004D0040E005CE3
:10407000000E01581DE302016B0E366F020E376F02
:104080005EEC29F002016C0E366F020E376F5EECAB
:1040900029F002016D0E366F020E376F5EEC29F0CB
:1040A00002016E0E366F020E376F5EEC29F001D002
:1040B000CAD0040E04010B5F04010B510B07000969
:1040C00008E002010C0E366F040E376F5EEC29F02B
:1040D000F3D787D002010B0E366F040E376F5EECFC
:1040E00029F004010B51006E016A040E001801E171
:1040F00001501DE10201120E366F040E376F5EECA7
:1041000029F00201110E366F040E376F5EEC29F0B4
:104110000201100E366F040E376F5EEC29F00201BB
:104120000F0E366F040E376F5EEC29F001D08BD086
:1041300058D0010E0E6F55D002010B0E366F040ED3
:10414000376F5EEC29F004010B51006E016A040E1A
:10415000001801E101502FE10201660E366F020ED8
:10416000376F5EEC29F00201650E366F020E376F75
:104170005EEC29F00201640E366F020E376F5EECC2
:1041800029F00201630E366F020E376F5EEC29F0E4
:10419000080ED88002016355070E6455000E655560
:1041A000000E665507E2080E635F070E645B000EA3
:1041B000655B665B01D047D014D002010B0E366FF1
:1041C000040E376F5EEC29F004010B510B07000958
:1041D00008E002010C0E366F040E376F5EEC29F01A
:1041E000F3D70EC400F0016A00BE01680050011050
:1041F00001E1B5D604010D51006E016A020E0018EE
:1042000001E1015009E10FC45FF210C460F211C472
:1042100061F212C462F212D05F0EE96E020EEA6E13
:10422000EE500F1909E1EE50101906E1EE50111988
:1042300003E1EE50121900E101E00D6BCAEC29F028
:1042400004010D5104D0CAEC29F0000E00D0120078
:104250000201010E346F37EC28F00201010E346FB9
:1042600037EC28F00201060E346F37EC28F002011B
:10427000346B37EC28F00201120E346F37EC28F063
:104280000201230E346F37EC28F00201340E346F34
:1042900037EC28F00201560E346F37EC28F002019B
:1042A000346B37EC28F00201346B37EC28F0020154
:1042B000800E346F37EC28F00201346B37EC28F0B5
:1042C0000201346B37EC28F00201346B37EC28F034
:1042D0000201346B37EC28F00201346B37EC28F024
:1042E0000401196B1951006E016A0150000AE8AE11
:1042F00002D0D89004D00C0E005C000E015807E2EA
:104300000201346B37EC28F00401192BEBD70001C4
:1043100084510201346F37EC28F00001855102010D
:10432000346F37EC28F0000186510201346F37EC0E
:1043300028F0000187510201346F37EC28F00001AA
:1043400088510201346F37EC28F0000189510201D5
:10435000346F37EC28F00401196B1951006E016AB3
:104360000150000AE8AE02D0D89004D0CA0E005C1A
:10437000000E015807E20201346B37EC28F004010B
:10438000192BEBD70201630E346F37EC28F00201D2
:10439000820E346F37EC28F00201530E346F37EC85
:1043A00028F00201630E346F37EC28F00201350E5D
:1043B000346F37EC28F00201010E346F37EC28F02F
:1043C000020177510201346F37EC28F00201775176
:1043D000026E036A010E021801E1035005E0675105
:1043E000681169116A1102E1000E01D0010E006E20
:1043F000016A0050011022E00201360E346F37ECE2
:1044000028F00201040E346F37EC28F002016251EB
:104410000201346F37EC28F0020161510201346F60
:1044200037EC28F0020160510201346F37EC28F0BC
:1044300002015F510201346F37EC28F00201370EA0
:10444000346F37EC28F00201020E346F37EC28F09D
:104450000201010E346F37EC28F00201030E346FB5
:1044600037EC28F002017751006E016A030E001844
:1044700001E1015022E10201320E346F37EC28F0E5
:104480000201040E346F37EC28F00201675102017B
:10449000346F37EC28F0020168510201346F37ECB9
:1044A00028F0020169510201346F37EC28F0020153
:1044B0006A510201346F37EC28F00201346937EC9D
:0644C00028F0B7EF28F020
:0A44C6000401006B0051006E016A52
:1044D000010E005C000E015825E20051040DF3CFDF
:1044E00000F0F4CF01F0400E0026000E0122005132
:1044F000E96EEA6AD890E936EA36D70EE926010E67
:10450000EA2200C0EFFF0051E96EEA6AD890E9366E
:10451000EA36D70EE926010EEA22EE52010EEF6EC0
:10452000002BD3D70101DB6BDCEC26F00A0EE66E24
:104530009FEC3DF0E55201011F0EF26FF8EC26F002
:104540000101F16F01011F0EF06FECEC26F00A0E75
:10455000E66E9FEC3DF0E5520101070EF26FF8ECBC
:1045600026F0006E016A0050800B01E1CCD0010101
:10457000210EF16F0101F06BECEC26F00A0EE66EF5
:104580009FEC3DF0E5520101480EF16F01010E0E66
:10459000F06FECEC26F00101F16B01010A0EF06FF7
:1045A000ECEC26F00101F16B01010B0EF06FECEC6D
:1045B00026F00101040EF16F01010C0EF06FECEC1E
:1045C00026F00101020EF16F01010D0EF06FECEC0F
:1045D00026F00101DB51E96EEA6AD890E936EA3645
:1045E000D70EE926010EEA22EF500101F16F010119
:1045F000040EF06FF1DB0101440EF16F0101010EB9
:10460000F06FEADB01015F0EF16F0101020EF06F46
:10461000E3DB01015E0EF16F0101030EF06FDCDBE5
:104620000101F1690101070EF06FD6DB0101F16BA9
:1046300001010F0EF06FD0DB0101610EF16F01017E
:10464000F06BCADB000184510101F16F0101010E21
:10465000F06FC2DB000185510101F16F0101020E13
:10466000F06FBADB000186510101F16F0101030E09
:10467000F06FB2DB000187510101F16F0101040EFF
:10468000F06FAADB000188510101F16F0101050EF5
:10469000F06FA2DB000189510101F16F0101060EEB
:1046A000F06F9ADB0401006B0051006E016A01504B
:1046B000000AE8AE02D0D89004D0080E005C000ECC
:1046C00001580BE20101F169080E04010025010106
:1046D000F06F82DB0401002BE7D70101440EF16F7C
:1046E0000101070EF06F78DB0101440ED96F010163
:1046F000220EF16F0101F06B6FDB0101F16B010123
:104700000D0EF06F69DB12000101F26B71DB026EBE
:10471000036A0250040B02E0000E01D0010E006E8D
:10472000016A005000D012000101010EF16F010179
:104730000A0EF06F51DB0101F16B01010B0EF06FFE
:104740004BDB0101120EF16F0101F06B45DB010142
:10475000DC510101F16F0101100EF06FECEF26F05A
:10476000010E0101DF15006E016ADF510024040112
:10477000A26F0101E05101200401A36F0101400E6D
:10478000F16F0101070EF06F27DB0401A251010157
:10479000F16F01010A0EF06F1FDB0401A35101014B
:1047A000F16F01010B0EF06F17DB0101120EF16FBB
:1047B0000101F06B11DB0101DFC100F0E0C101F08C
:1047C000DF07000EE05BD8800054000E01540FE2BA
:1047D000DDC1E9FFDEC1EAFFDD2B000EDE23EF5075
:1047E0000101F16F0101100EF06FF6DAE4D7DF6915
:1047F000E06BDF51E01109E00101070EF26FF8DA1A
:10480000026E036A0250400B02E0000E01D0010E5E
:10481000006E016A0050011005E00101DF07000E83
:10482000E05BE7D712000101010EF16F01010A0EF2
:10483000F06FD2DA0101F16B01010B0EF06FCCDAEF
:1048400001010A0EF16F0101F06BC6DA0101100ED1
:10485000F26FCEDA00D01200E3C131F4E4C132F4D9
:104860000101400EF16F0101070EF06FB5DA04018E
:1048700031510101F16F01010A0EF06FADDA04014F
:1048800032510101F16F01010B0EF06FA5DA010148
:104890000A0EF16F0101F06B9FDA0101E3C100F034
:1048A000E4C101F0E307000EE45BD8800054000E81
:1048B000015411E20101100EF26F9ADAE66E010165
:1048C000E1C1E9FFE2C1EAFFE12B000EE223E5527C
:1048D000E750EF6EE2D731C4F3FF32C4F4FF00D0EB
:1048E00012000101E551E96EEA6AD890E936EA362C
:1048F000D70EE926010EEA22EE52EF6A12000101FC
:10490000E651E96EEA6AD890E936EA36D70EE9262A
:10491000010EEA22EE52010EEF6EE651DB6F12003D
:104920000101D951006E016A0006000E015A00C053
:1049300067F404016751006E016A0150000AE8AE95
:1049400002D0D89004D0440E005C000E015802E260
:104950005E0E676F0101200EF16F0101F06B3CDA12
:10496000040167510101F16F0101030EF06F34DAA8
:1049700000D012000101600EF16F0101F06B2CDA22
:104980000101070EF26F34DA04018B6F0101200E72
:10499000F16F0101F06B20DA04018B51006E016AA6
:1049A0000101DA51000101AF02D0D89003D0005DBF
:1049B000000E015911E20101DA51006E016A5F0E29
:1049C000D8800056000E015604018B51026E036A16
:1049D000005002248C6F10D004018B51026E036AC8
:1049E0000101DA51046E056A0450025C006E055044
:1049F0000358016E00C08CF404018C51006E016AF2
:104A00001B0ED8800056000E015600C08CF48C514D
:104A10008E6F8D6B8DC4F3FF8EC4F4FF00D0120037
:104A20000101E00EF16F0101F06BD6D90101030E17
:104A3000F26FDED90401006F0101200EF16F010158
:104A4000F06BCAD904010051040B01E0010E026EA3
:104A5000036A0250031002E0000E01D0010E006E46
:104A6000016A005000D01200E9C1E9FFEAC1EAFF83
:104A7000EF680101070EF26FBBD9006E016A0050AA
:104A8000100B31E00101210EF16F0101F06BA4D98F
:104A90000101F569D7D90101F16B01010A0EF06F2F
:104AA0009BD90101F16B01010B0EF06F95D901014A
:104AB000020EF16F01010D0EF06F8ED90101200E73
:104AC000F16F0101F06B88D92BDF0101F169010160
:104AD000070EF06F81D90101F16B01010D0EF06F2E
:104AE0007BD9000EB2D00101600EF16F0101F06BB5
:104AF00073D90101070EF26F7BD90401126F010116
:104B0000200EF16F0101F06B67D904011251006EA4
:104B1000016A0101D951026E036A0250001802E1D4
:104B20000350011801E18FD0D9510401146F136BA8
:104B300013C4F3F114C4F4F169D9120E0101E36F47
:104B4000E46B0101000EE16F040EE26F85DE0401EB
:104B50000051010B046E056A0450051005E0400E7B
:104B6000025D000E035902E2000E01D0010E026E3A
:104B7000036A0250031006E0EE0ED8800255050EBF
:104B8000035502E2000E01D0010E006E016A0050D2
:104B9000011050E010C4C8F211C4C9F2FFEC37F0A4
:104BA000F3CF10F4F4CF11F4060EE66EE66A0A0EA7
:104BB000E66E040EE66EE7C1E9FFE8C1EAFFE9CF61
:104BC00000F0EACF01F000C0E6FF01C0E6FF28ECEC
:104BD0003BF0F56E060EE15EF55004011151026ED8
:104BE000036A080E021801E1035016E11051066E27
:104BF000076A065007100AE01051086E096A060E8F
:104C0000081801E1095002E0000E01D0010E046E07
:104C1000056A0450051002E1000E01D0010E006E7D
:104C2000016A0050011006E01051E9C1E9FFEAC134
:104C3000EAFFEF6E0101D951DA6F04010151010160
:104C4000D96F010E02D0000E00D0120001010A0E31
:104C5000F16F0101070EF06FBFD80101DB51E96E62
:104C6000EA6AD890E936EA36D70EE926010EEA223A
:104C7000EF500401A06F9F6B9FC4F3F1A0C4F4F147
:104C8000C5D8060E0101DF6FE06BEBC1DDF1ECC1B1
:104C9000DEF166DD000184510101DC6F45DD0001BC
:104CA00085510101DC6F40DD000186510101DC6F9F
:104CB0003BDD000187510101DC6F36DD00018851C9
:104CC0000101DC6F31DD000189510101DC6F2CDD58
:104CD0000101ED51006E016A0050011003E1040171
:104CE000A16B03D00401060EA16F0101080EDC6F59
:104CF0001BDD0401A1510101DC6F16DD0E0E010167
:104D0000EE27000EEF233C0EEE5D000EEF5903E29E
:104D1000400EEE6FEF6BEEC19FF4EFC1A0F4040103
:104D20009F510101F16F0101050EF06F55D804018B
:104D3000A0510101F16F0101060EF06FECEF26F0BA
:104D40000101DB51E96EEA6AD890E936EA36D70EFE
:104D5000E926010EEA22EF500101F16F0101040E74
:104D6000F06F3AD80101240EF16F0101F06B34D8D5
:104D700004018B6B8B51006E016A010E005C000E0A
:104D8000015819E28B51E96EEA6AD890E936EA36A1
:104D9000D70EE926010EEA22EE52EFCF00F0016AAB
:104DA00000BE01680050011004E08B510101DB6F6F
:104DB00002D08B2BDFD712009568816AE00E936ECC
:104DC000F19E848284808484966A050EE66EBDEC32
:104DD0003DF0E552849412000101F051816EE00E25
:104DE000936EF151836E956A849284829568120065
:104DF00095680101F251816EE00E936E84908350AC
:104E00000401A46F8480A45100D01200F3C1A2F465
:104E1000F4C1A3F40101400EF16F0101070EF06F20
:104E2000DBDF0401A2510101F16F0101080EF06FF7
:104E3000D3DF0401A3510101F16F0101090EF06FED
:104E4000ECEF26F00101F5510401166F156B15C446
:104E500000F016C401F01507000E165BD880005450
:104E6000000E015401E2F3D712000101DA510401EE
:104E7000686F120E676F0101F65104016727010187
:104E8000F7510401682367C4F3F168C4F4F106EF35
:104E900027F00101F851DB6FDB51E96EEA6AD89027
:104EA000E936EA36D70EE926010EEA22EF50040170
:104EB0008C6F0E0E8B6F0101F95104018B270101DC
:104EC000FA5104018C238BC4F3F18CC4F4F106EF86
:104ED00027F00101090EF26F8BDF0401016F010160
:104EE000080EF26F85DF0401006F00C4F3FF01C4F8
:064EF000F4FF00D01200E7
:0A4EF6000401006B0051006E016A18
:104F00000150000AE8AE02D0D89004D0020E005C36
:104F1000000E015821E20051160DF3CFE9FFF4CF46
:104F2000EAFF000EE926020EEA220C0EE926000E28
:104F3000EA22EE6AED6A0051160DF3CFE9FFF4CFD5
:104F4000EAFF000EE926020EEA22150EE926000EFF
:104F5000EA22EF90002BD1D712000401000E0C6F53
:104F6000020E0D6F0B6B0B51006E016A0150000AAF
:104F7000E8AE02D0D89004D0020E005C000E0158BA
:104F800061E20CC4E9FF0DC4EAFF0C0EE926000E35
:104F9000EA22EECF00F0EFCF01F0026A036A005080
:104FA00001100210031048E10CC4E9FF0DC4EAFF30
:104FB0000C0E2DC2EBFF0D0E2EC2EBFF02012F5186
:104FC000301119E00A0EE66EE66A2FC2E6FF30C223
:104FD000E6FF0CC4E9FF0DC4EAFFE9CF00F0EACF19
:104FE00001F000C0E6FF01C0E6FF28EC3BF0F56EE3
:104FF000060EE15EF5500CC4E9FF0DC4EAFF0A0E8F
:1050000031C2EBFF0B0E32C2EBFF0CC4E9FF0DC443
:10501000EAFF0E0EEB6A0F0EEB6A0CC4E9FF0DC43B
:10502000EAFF100EEB6A110EEB6A04010B5102014C
:105030002C6F04010B5108D0160E0C27000E0D2307
:105040000B2B91D7FF0E00D0120002013351160D29
:10505000F3CFE9FFF4CFEAFF000EE926020EEA22C1
:105060000C0EE926000EEA22EE6AED6A1200020139
:105070002C51160DF3CF15F4F4CF16F4000E0401E5
:105080001527020E162315C4E9FF16C4EAFF0E0EFB
:10509000E926000EEA22EE50ED1024E10101DB5179
:1050A000E66E15C4E9FF16C4EAFF120EE926000EEB
:1050B000EA22E552E750EF6E1C0E0101F96FFA6B20
:1050C00015C4E9FF16C4EAFF120EEB500101F86F98
:1050D00049EC27F015C4E9FF16C4EAFF130EEB6A8A
:1050E000140EEB6A020134510101DC6F94EC23F0E1
:1050F00015C4E9FF16C4EAFF130EE926000EEA22E2
:10510000EECF00F0EDCF01F0EE2AEF2215C4E9FF5B
:1051100016C4EAFF0E0EE926000EEA22EECF02F0D8
:10512000EFCF03F00250005C035001580AE315C4AE
:10513000E9FF16C4EAFF0E0EE926000EEA22EE2A67
:10514000EF2215C4E9FF16C4EAFF0E0EE926000E91
:10515000EA22EECF17F4EDCF18F40401D60E175D56
:10516000030E185901E303D8010E00D0120002010A
:105170002C51160DF3CF13F4F4CF14F4000E0401E8
:105180001327020E142313C4E9FF14C4EAFF0C0E04
:10519000E926000EEA22EECFC8F2EDCFC9F2FFEC0D
:1051A00037F0F3CF0BF4F4CF0CF413C4E9FF14C4BD
:1051B000EAFF0A0EE926000EEA22EECFC8F2EDCF92
:1051C000C9F2FFEC37F0F3CF0DF4F4CF0EF413C4B3
:1051D000E9FF14C4EAFF0E0EE926000EEA22EECF24
:1051E0000FF4EFCF10F4080E04010F27000E102368
:1051F000116B126B140E0101F96FFA6B13C4E9FF06
:1052000014C4EAFF120EEB500101F86F49EC27F0CD
:105210000FC4AEF210C4AFF20201110EAD6F13C491
:10522000E9FF14C4EAFFE9CFABF2EACFACF255ECE8
:1052300032F00FC4C8F210C4C9F2FFEC37F0F3CF5C
:105240000FF4F4CF10F4080E0101DF6FE06B0101E1
:105250000B0EDD6F040EDE6FB0EC23F0A0EC26F039
:1052600013C4E9FF14C4EAFF120EE926000EEA2275
:10527000EF6813C4E9FF14C4EAFF0E0EEB6A0F0EC9
:10528000EB6A1200020135512C6F2C51160DF3CF31
:10529000E9FFF4CFEAFF000EE926020EEA22100E23
:1052A000E926000EEA22D880EE54000EED54D870A4
:1052B000006A016A0036005000D0120002012C5131
:1052C000160DF3CFE9FFF4CFEAFF000EE926020E38
:1052D000EA22100EE926000EEA22EE50ED1002E15D
:1052E000000E57D02C51160DF3CFE9FFF4CFEAFF93
:1052F000000EE926020EEA22150EE926000EEA2229
:10530000EF50010B006E016A0050011015E02C51A6
:10531000160DF3CFE9FFF4CFEAFF000EE926020EE7
:10532000EA22150EE926000EEA22EF901C0E01017A
:10533000F66FF76B35EC27F013EC24F036C2E9FF7B
:1053400037C2EAFFEF6E02012C51160DF3CFE9FFD1
:10535000F4CFEAFF000EE926020EEA22100EE9263B
:10536000000EEA22EE06EF5A2C51160DF3CFE9FF9C
:10537000F4CFEAFF000EE926020EEA22100EE9261B
:10538000000EEA22EE50ED1002E190EC24F0010E46
:1053900000D0120002012C51160DF3CFE9FFF4CF1B
:1053A000EAFF000EE926020EEA22100EE926000EA0
:1053B000EA22EE50ED1002E090EC24F002012C51B4
:1053C000160DF3CFE9FFF4CFEAFF000EE926020E37
:1053D000EA22100EE926000EEA22EE6AED6A1200B9
:1053E000080E0101E36FE46B0101000EE16F040E92
:1053F000E26F2CEC24F000C4C8F201C4C9F2FFEC47
:1054000037F0F3CF00F4F4CF01F402C4C8F203C4C0
:10541000C9F2FFEC37F0F3CF02F4F4CF03F404C485
:10542000C8F205C4C9F2FFEC37F0F3CF04F4F4CFAF
:1054300005F40401080E045F000E055B06C4C8F203
:1054400007C4C9F2FFEC37F0F3CF06F4F4CF07F44A
:1054500038C23EF239C23FF20201000E3C6F040E28
:105460003D6F31D80401086F0851006E016AFF0ECC
:10547000001801E1015003E190EC24F021D0085123
:10548000160DF3CFE9FFF4CFEAFF000EE926020E76
:10549000EA22100EE926000EEA2204C4EEFF05C43B
:1054A000EDFF0851160DF3CFE9FFF4CFEAFF000E30
:1054B000E926020EEA22150EE926000EEA22EF8006
:1054C000010E00D0120004010A69000E0B6F020EDB
:1054D0000C6F096B0951006E016A0150000AE8AEB9
:1054E00002D0D89004D0020E005C000E015801E3F7
:1054F000A2D00BC4E9FF0CC4EAFF0C0EE926000E93
:10550000EA22EECF00F0EFCF01F03CC2E9FF3DC24E
:10551000EAFF020EE926000EEA22EECF02F0EFCFFC
:1055200003F00250001802E10350011801E07DD0A1
:105530000BC4E9FF0CC4EAFF0A0EE926000EEA22BA
:10554000EECF02F0EFCF03F03CC2E9FF3DC2EAFF2D
:10555000EECF04F0EFCF05F00450021802E1055041
:10556000031813E10BC4E9FF0CC4EAFF100EE9268F
:10557000000EEA22EECF06F0EFCF07F0086A096AC4
:10558000065007100810091002E0000E01D0010EAD
:10559000006E016A0050011045E03EC2E9FF3FC2C3
:1055A000EAFF060EE926000EEA22EECF02F0EECF69
:1055B00003F0EECF04F0EFCF05F00BC4E9FF0CC40D
:1055C000EAFF060EE926000EEA22EE50000102195B
:1055D00009E1EE50031906E1EE50041903E1EE5023
:1055E000051900E116E00BC4E9FF0CC4EAFF060E42
:1055F000E926000EEA22E868EE1808E1E868EE18ED
:1056000005E1E868EE1802E1E868EE1802E0000E35
:1056100001D0010E006E016A0050011003E0040188
:10562000095149D0040109510A6F160E0B27000ECB
:105630000C23092B4FD70A51006E016AFF0E001888
:1056400001E1015035E00A51160DF3CF0BF4F4CF10
:105650000CF4000E0B27020E0C230A0EE66EE66A0F
:105660003EC2E6FF3FC2E6FF0BC4E9FF0CC4EAFFFF
:10567000E9CF00F0EACF01F000C0E6FF01C0E6FF8D
:1056800028EC3BF0F56E060EE15EF5503CC2E9FFFA
:105690003DC2EAFFEECF00F0EFCF01F00BC4E9FF0F
:1056A0000CC4EAFF0A0E00C0EBFF0B0E01C0EBFFBB
:0856B00004010A5100D01200B0
:0856B8003C68746D6C3E3C6817
:1056C0006561643E3C7469746C653E576562205345
:1056D000657276657220492F4F20436F6E74726F2A
:1056E0006C3C2F7469746C653E3C2F686561643E48
:1056F0003C626F64793E3C63656E7465723E3C66E5
:105700006F6E7420666163653D68656C766574696B
:1057100063613E3C68323E3C753E4F7574707574F3
:1057200020436F6E74726F6C3C2F753E3C2F683255
:105730003E3C464F524D204D4554484F443D474511
:105740005420616374696F6E3D303E3C7461626CDD
:105750006520626F726465723D323E3C74723E3CFD
:1057600074643E3C696E70757420747970653D7325
:1057700075626D6974206E616D653D312076616C76
:1057800075653D44363D2530313E3C2F74643E3CCA
:1057900074643E3C696E70757420747970653D73F5
:1057A00075626D6974206E616D653D302076616C47
:1057B00075653D44353D2530303E3C2F74643E3C9C
:1057C0002F74723E3C2F7461626C653E3C2F666F95
:1057D000726D3E3C2F626F64793E3C2F68746D6C35
:1057E0003E04FFFFFF3C48544D4C3E3C484541447D
:1057F0003E3C5449544C453E4D6963726F63686941
:1058000070205443502F495020537461636B2044DF
:10581000656D6F3C2F5449544C453E3C2F484541E3
:10582000443E3C4652414D4553455420726F777378
:105830003D223130302C33302220626F7264657229
:105840003D303E20203C4652414D45206E616D6505
:105850003D22746F702220097372633D226D61696D
:105860006E2E68746D22206D617267696E6865695D
:105870006768743D35206D617267696E776964741D
:10588000683D353E093C4652414D455345542063E1
:105890006F6C733D2238302C38302220626F726476
:1058A00065723D303E202009093C4652414D45205D
:1058B0006E616D653D226C656674222020207372D6
:1058C000633D225374617475732E63676922206D82
:1058D000617267696E6865696768743D32206D61E1
:1058E0007267696E77696474683D323E20200909E9
:1058F0003C4652414D45206E616D653D227269679F
:105900006874222020207372633D22436F6D6D61A5
:105910006E64732E63676922206D617267696E68B9
:1059200065696768743D32206D617267696E776979
:105930006474683D323E093C2F4652414D45534503
:10594000543E3C2F4652414D455345543E3C2F4812
:10595000544D4C3E04FFFFFF3C48544D4C3E3C48E8
:105960004541443E3C2F484541443E3C424F44590A
:105970003E3C666F6E7420666163653D68656C765B
:1059800065746963613E3C63656E7465723E3C425A
:105990003E3C553E3C464F4E542053495A453D37B8
:1059A00020434F4C4F523D22233030303066662228
:1059B0003E3C503E4D6963726F636869702054438A
:1059C000502F495020537461636B3C2F503E3C2F45
:1059D000423E3C2F553E3C2F464F4E543E3C2F639B
:1059E000656E7465723E5468697320697320612026
:1059F00073616D706C65207061676520696E746598
:105A00006E64656420746F2064656D6F6E7374726C
:105A1000617465204D6963726F63686970205443D7
:105A2000502F495020537461636B20636170616231
:105A3000696C69746965732E546869732070616755
:105A400065206973207365727665642062792048E9
:105A5000545450205365727665722C2072756E6EA8
:105A6000696E67206F6E204D6963726F636869703D
:105A7000205049433138206D6963726F636F6E74D3
:105A8000726F6C6C65722C7574696C697A696E677B
:105A9000204D6963726F63686970205443502F49C9
:105AA0005020537461636B2E3C703E4D6963726F7E
:105AB0006368697020537461636B206F66666572FA
:105AC0007320666F6C6C6F77696E672066656174B2
:105AD000757265733A3C2F703E3C756C3E3C6C6948
:105AE0003E506F727461626C65206163726F737394
:105AF000204D6963726F6368697020504943313883
:105B00002066616D696C79206F66206D6963726FC4
:105B1000636F6E74726F6C6C6572733C2F6C693E50
:105B20003C6C693E436F6F70657261746976652085
:105B30006D756C74697461736B696E672054435042
:105B40002F495020737461636B3C2F6C693E3C6C31
:105B5000693E5573652069742061732070617274A9
:105B6000206F662048545450205365727665722029
:105B70006F7220637573746F6D205443502F4950BA
:105B8000206261736564206170706C69636174691F
:105B90006F6E3C2F6C693E3C6C693E4D756C746950
:105BA000706C652054435020736F636B6574207371
:105BB0007570706F72743C2F6C693E3C6C693E4826
:105BC000545450205365727665722077697468204A
:105BD0006D756C7469706C6520636F6E6E6563744F
:105BE000696F6E7320737570706F72743C2F6C697F
:105BF0003E3C6C693E5061676573206D617920623F
:105C0000652073746F72656420696E20696E7465B7
:105C1000726E616C2070726F6772616D206D656D60
:105C20006F7279206F722065787465726E616C2076
:105C30006461746120454550524F4D3C2F6C693E64
:105C40003C6C693E537570706F727420666F722081
:105C500048544D4C20666F726D733C2F6C693E3C0E
:105C60006C693E50432062617365642070726F6797
:105C700072616D20746F20636F6E76657274207729
:105C8000656220706167657320696E746F204D696D
:105C900063726F636869702046696C65205379731D
:105CA00074656D20284D504653293C2F6C693E3C4D
:105CB0006C693E4D6F64756C6172206465736967D1
:105CC0006E20746F20656173696C79206164642053
:105CD0006E657720636F6D706F6E656E74733C2FA9
:105CE0006C693E3C2F756C3E3C2F424F44593E3C04
:105CF0002F48544D4C3E04FFFFFF3C68746D6C3ED2
:105D00003C6D65746120687474702D657175697679
:105D10003D22726566726573682220636F6E7465DA
:105D20006E743D2233223E3C686561643E3C74697A
:105D3000746C653E576562205365727665722053B8
:105D400074617475733C2F7469746C653E3C2F6884
:105D50006561643E3C626F64793E3C63656E746568
:105D6000723E3C666F6E7420666163653D68656C6B
:105D70007665746963613E3C753E3C68323E53799A
:105D80007374656D205374617475733C2F68323E73
:105D90003C2F753E3C7461626C6520626F72646575
:105DA000723D323E3C74723E3C74643E53333D253A
:105DB00030343C2F74643E3C74643E44363D2530A0
:105DC000313C2F74643E3C74643E44353D25303094
:105DD0003C2F74643E3C74643E414E303D2530326D
:105DE0003C2F74643E3C74643E414E313D2530335B
:105DF0003C2F74643E3C2F74723E3C2F7461626C85
:105E0000653E3C62723E3C2F626F64793E3C2F6877
:105E1000746D6C3E04FFFFFF00B856434F4D4D417B
:105E20004E44532E43474900E557494E4445582EAA
:105E300048544D2020200058594D41494E2E485479
:105E40004D2020202000FA5C5354415455532E43DA
:105E50004749202004FFFF454E44204F462046413D
:035E6000542020AB
:0C5E64001C0E0101E36FE46B0101000E55
:105E7000E16F040EE26F2CEC24F090EC24F00001B2
:105E8000000EFE6F040EFF6FC3D90401010E00194E
:105E900001E101510AE10451046E056A060E04187D
:105EA00001E1055002E1000E01D0010E026E036A0D
:105EB000025003100AE10551066E076A040E061827
:105EC00001E1075002E1000E01D0010E006E016AEF
:105ED0000050011002E0000E93D0020E061901E1FD
:105EE000075106E1F9C0E9FFFAC0EAFFEF6A14D0F2
:105EF000010E061901E1075107E1010EF9C0E9FFA2
:105F0000FAC0EAFFEF6E08D0020EF9C0E9FFFAC04E
:105F1000EAFFEF6E000E74D01851066E076A00019A
:105F20008051086E096A0850061802E109500718E6
:105F30000EE1040119510A6E0B6A000181510C6EC9
:105F40000D6A0C500A1802E10D500B1802E0000E09
:105F500001D0010E046E056A045005100EE0040124
:105F60001A510E6E0F6A00018251106E116A1050A4
:105F70000E1802E111500F1802E0000E01D0010EC0
:105F8000026E036A025003100EE004011B51126EF0
:105F9000136A00018351146E156A1450121802E13D
:105FA0001550131802E0000E01D0010E006E016AB8
:105FB0000050011023E0F7C0E9FFF8C0EAFF08C471
:105FC000EEFF09C4EEFF0AC4EEFF0BC4EEFF0CC4E3
:105FD000EEFF0DC4EEFFF7C0E9FFF8C0EAFF060EC2
:105FE000E926000EEA220EC4EEFF0FC4EEFF10C435
:105FF000EEFF11C4EEFF010E03D002D0000E00D060
:106000001200010E0401006F016B026B080E036F9A
:10601000060E046F040E056F0001FD51006E016A4B
:10602000010E001801E101500BE1010E0401066FA1
:10603000076B12691369146915691669176914D019
:10604000020E0401066F076BFBC0E9FFFCC0EAFF0C
:10605000EECF12F4EECF13F4EECF14F4EECF15F42E
:10606000EECF16F4EFCF17F4000184510401086F4E
:10607000000185510401096F0001865104010A6F76
:106080000001875104010B6F0001885104010C6F5E
:106090000001895104010D6F0001805104010E6F50
:1060A0000001815104010F6F000182510401106F42
:1060B000000183510401116FFBC0E9FFFCC0EAFF3E
:1060C000060EE926000EEA22EF500E1900018A158D
:1060D000066E076A0650071018E1FBC0E9FFFCC016
:1060E000EAFF060EE926000EEA22010EE926000E5E
:1060F000EA22EF5004010F1900018B15086E096A9E
:106100000850091002E1000E01D0010E046E056A6C
:106110000450051018E1FBC0E9FFFCC0EAFF060EC1
:10612000E926000EEA22020EE926000EEA22EF50CE
:106130000401101900018C150A6E0B6A0A500B102D
:1061400002E1000E01D0010E026E036A025003103C
:1061500018E1FBC0E9FFFCC0EAFF060EE926000ECD
:10616000EA22030EE926000EEA22EF50040111197B
:1061700000018D150C6E0D6A0C500D1002E1000E21
:1061800001D0010E006E016A0050011010E08E5126
:106190000401186F00018F510401196F0001905123
:1061A00004011A6F0001915104011B6F10D0FBC054
:1061B000E9FFFCC0EAFF060EE926000EEA22EECF58
:1061C00018F4EECF19F4EECF1AF4EFCF1BF4000160
:1061D000000EFE6F040EFF6F1BD81C0E0101EE6F48
:1061E000EF6B0101060EED6F0101120EEB6F040E55
:1061F000EC6F26EC26F01C0E0101DF6FE06B010155
:10620000000EDD6F040EDE6FB0EC23F0A0EF26F081
:10621000FEC0E9FFFFC0EAFFEECFC8F2EDCFC9F242
:10622000FFEC37F0F3CF00F0F4CF01F0FEC0E9FF50
:10623000FFC0EAFF00C0EEFF01C0EDFFFEC0E9FFB6
:10624000FFC0EAFF020EE926000EEA22EECFC8F2F6
:10625000EDCFC9F2FFEC37F0F3CF00F0F4CF01F04F
:10626000FEC0E9FFFFC0EAFF020E00C0EBFF030E15
:1062700001C0EBFFFEC0E9FFFFC0EAFF060EE92602
:10628000000EEA22EECFC8F2EDCFC9F2FFEC37F0F4
:10629000F3CF00F0F4CF01F0FEC0E9FFFFC0EAFF4A
:0E62A000060E00C0EBFF070E01C0EBFF120060
:0262AE00140ECC
:1062B0000101E36FE46B0101080EE16F040EE26F70
:1062C0002CEC24F0F00E04010815006E016A400E5B
:1062D000001801E1015001E0E3D00F0E0815006E37
:1062E000016AD89000360136D89000360136140E77
:1062F000005E000E015A00C01CF41C51006E016AC1
:106300000150000AE8AE02D0013405D0140ED88046
:106310000054000E015401E2C3D01C51006E016A0A
:106320000150000AE8AE02D0013405D0000ED8803A
:106330000054000E01540BE21C510101E36FE46BA9
:1063400001011D0EE16F040EE26F2CEC24F012C46B
:1063500000F413C401F40401126B136B140E020158
:10636000D06FD16B0201080ECE6F040ECF6F7EECA2
:1063700038F0F3CF04F4F4CF05F40401041F051F33
:106380001C51006E016A0150000AE8AE02D00134CF
:1063900005D0000ED8800054000E015413E21C51A9
:1063A0000201D06FD16B02011D0ECE6F040ECF6FB4
:1063B0007EEC38F0F3CF06F4F4CF07F40401061FA7
:1063C000071F02D0066B076B040E0201D06FD16B62
:1063D0000201040ECE6F040ECF6F7EEC38F0F3CFC7
:1063E00002F4F4CF03F40201080EB06F040EB16F93
:1063F000DBD804010251001902E1035101190BE13C
:10640000F00E0815026E036A400E021801E10350F7
:1064100002E1000E01D0010E006E016A0050011071
:1064200001E03ED00201A351A4110CE0A3C2E9FF98
:10643000A4C2EAFF18C4EEFF19C4EEFF1AC4EEFFAF
:106440001BC4EEFFA5C2E9FFA6C2EAFF060EE926BD
:10645000000EEA2214C4EEFF15C4EEFF16C4EEFFD0
:1064600017C4EEFF04011151A7C2E9FFA8C2EAFF59
:10647000EF6E1C51026E036A02500A5D006E0350FB
:106480000B59016E140E005E000E015AA9C2E9FFFD
:10649000AAC2EAFF00C0EEFF01C0EDFF010E04D06A
:1064A00090EC24F0000E00D012000401450E8B6F1A
:1064B0008C6B140E0201AE2504018D6F000E0201DB
:1064C000AF2104018E6F0201E42B000EE523E4C22C
:1064D0008FF4E5C290F40401916B926B640E936F9C
:1064E0000201AD510401946F956B966B00018051D0
:1064F0000401976F000181510401986F00018251DE
:106500000401996F0001835104019A6FABC2E9FF46
:10651000ACC2EAFF060EE926000EEA22EECF9BF49B
:10652000EECF9CF4EECF9DF4EFCF9EF402018B0EE4
:10653000B06F040EB16F38D8140E0201D06FD16B5A
:1065400002018B0ECE6F040ECF6F7EEC38F0F3CFCE
:1065500095F4F4CF96F4140E0201AE250101EE6F0E
:10656000000E0201AF210101EF6F0101ED6BABC223
:10657000E9FFACC2EAFFE9CFEBF1EACFECF126ECA0
:1065800026F0140E0101DF6FE06B01018B0EDD6F51
:10659000040EDE6FB0EC23F0006A016A00C0F3FF66
:1065A00001C0F4FF00D01200B0C2E9FFB1C2EAFF9F
:1065B000020EE926000EEA22EECFC8F2EDCFC9F2B4
:1065C000FFEC37F0F3CF00F0F4CF01F0B0C2E9FFF9
:1065D000B1C2EAFF020E00C0EBFF030E01C0EBFFE9
:1065E000B0C2E9FFB1C2EAFF040EE926000EEA22BA
:1065F000EECFC8F2EDCFC9F2FFEC37F0F3CF00F0E9
:10660000F4CF01F0B0C2E9FFB1C2EAFF040E00C04E
:10661000EBFF050E01C0EBFFB0C2E9FFB1C2EAFF1C
:106620000A0EE926000EEA22EECFC8F2EDCFC9F23B
:10663000FFEC37F0F3CF00F0F4CF01F0B0C2E9FF88
:10664000B1C2EAFF0A0E00C0EBFF0B0E01C0EBFF68
:02665000120036
:0E6652000001C56BC68163EC22F034EC3DF014
:106660007BEC27F082EF00F00401010E3C6F3CC48C
:1066700000F0016A00BE01680050011001E13FD145
:1066800004013C6BC5C000F0016A00BE0168040E45
:10669000001801E1015001E112D1030E001801E1DF
:1066A000015001E1CED0060E001801E1015001E1D8
:1066B000B6D0070E001801E1015001E19ED0020E94
:1066C000001801E101504FE0050E001801E10150F2
:1066D00042E0005001E1015006E0010E001801E126
:1066E000015001E00BD101013B0EE96F040EEA6F8E
:1066F0000101C70EE76F000EE86F34EC25F00009CA
:106700000EE110EC25F0000909E10001806B816BBE
:10671000826B836B0001C68142EC1DF0EFD0040157
:10672000010E3C6F3B51006E016A0050011004E104
:106730000001020EC56F0ED03B51006E016A060EBD
:10674000001801E1015004E10001050EC56F02D0FF
:1067500090EC24F0D3D03C6B37EC3DF0000902E024
:106760000001C56BCBD00201D10EA96F000EAA6F3C
:1067700002013B0EA76F040EA86F0201C70EA56FA2
:10678000000EA66F0201370EA36F040EA46F57EC24
:1067900031F000092DE00401010E3C6F3B51006E09
:1067A000016A010E001801E1015004E10001030E2D
:1067B000C56F1DD03B51006E016A060E001801E145
:1067C000015004E10001060EC56F11D03B51006E6F
:1067D000016A110E001801E1015004E10001070EE9
:1067E000C56F05D03C6B90EC24F00001C56B04D064
:1067F00090EC24F00001C56B81D0D1C03AF2D2C038
:106800003BF20201C70E386F000E396FF0EC29F031
:10681000000902E00001C56B04013C6B6FD0D1C0E0
:10682000B2F1D2C0B3F10101C70EB06F000EB16F6B
:106830009CEC06F0000902E00001C56B04013C6B12
:106840005DD00001C56B290ED880D155000ED25500
:1068500033E30201F50E806F000E816F0201F30E2B
:106860007E6F000E7F6F0201D10E7C6F000E7D6F78
:106870000201D30E7A6F000E7B6F02013B0E786F20
:10688000040E796F8EEC34F0000914E03BC400F084
:10689000016A00BE0168080E001801E1015007E11D
:1068A0000401010E3C6F0001040EC56F02D000010F
:1068B000C56B02D00001C56B90EC24F01FD084ECB6
:1068C00023F000091AE0F5C08AF2F6C08BF2F3C09B
:1068D00088F2F4C089F2D1C087F20201D30E856F2D
:1068E000000E866F0201846B0201C70E826F000EDC
:1068F000836F17EC35F00001C56B00D0B8D699EC6A
:1069000004F060EC1DF00101FD51010B006E016A05
:0C6910000050011002E00001C6911200CE
:04691C00080E01015F
:10692000E36FE46B0101000EE16F040EE26F2CECEB
:1069300024F002C42EF403C42FF40401026B036B91
:10694000080E0201D06FD16B0201000ECE6F040E53
:10695000CF6F7EEC38F0F3CF28F4F4CF29F40401A4
:10696000281F291F080E006E7CC2E9FF7DC2EAFFC6
:106970000050EF5E7CC2E9FF7DC2EAFFEF500101EB
:10698000E36FE46B7AC2E1F17BC2E2F12CEC24F01C
:106990007CC2E9FF7DC2EAFFEF500201D06FD16BEC
:1069A0007AC2CEF27BC2CFF27EEC38F0F3CF2AF47B
:1069B000F4CF2BF404012A1F2B1F040E0201D06F09
:1069C000D16B0201280ECE6F040ECF6F7EEC38F033
:1069D000F3CF2CF4F4CF2DF40201000E8C6F040ED3
:1069E0008D6F85D80401005178C2E9FF79C2EAFFB2
:1069F000EF6E7EC2E9FF7FC2EAFF04C4EEFF05C46A
:106A0000EDFF80C2E9FF81C2EAFF06C4EEFF07C4C2
:106A1000EDFF2E512C1902E12F512D1902E0000E2D
:106A200001D0010E006E016A005000D01200040176
:106A3000016B84C200F0016A00BE016800C000F46E
:106A4000026B036B88C204F489C205F48AC206F49F
:106A50008BC207F402018751E66EE66A85C2E6FF43
:106A600086C2E6FF080EE66E040EE66E28EC3BF0EA
:106A7000F56E060EE15EF5500201000E8C6F040EFD
:106A80008D6F35D8080E020187250201D06FD16BBA
:106A9000000ED1230201000ECE6F040ECF6F7EECEC
:106AA00038F0F3CF02F4F4CF03F4080E0201872587
:106AB0000201AE6FAF6B000EAF230201010EAD6F8E
:106AC00082C2ABF283C2ACF255EC32F0080E020186
:106AD00087250101DF6FE06B000EE0230101000E4E
:106AE000DD6F040EDE6FB0EC23F0A0EF26F08CC259
:106AF000E9FF8DC2EAFF040EE926000EEA22EECF7E
:106B0000C8F2EDCFC9F2FFEC37F0F3CF00F0F4CFCD
:106B100001F08CC2E9FF8DC2EAFF040E00C0EBFF5A
:106B2000050E01C0EBFF8CC2E9FF8DC2EAFF060E25
:106B3000E926000EEA22EECFC8F2EDCFC9F2FFEC53
:106B400037F0F3CF00F0F4CF01F08CC2E9FF8DC233
:106B5000EAFF060E00C0EBFF070E01C0EBFF8CC280
:106B6000E9FF8DC2EAFF020EE926000EEA22EECF0F
:106B7000C8F2EDCFC9F2FFEC37F0F3CF00F0F4CF5D
:106B800001F08CC2E9FF8DC2EAFF020E00C0EBFFEC
:086B9000030E01C0EBFF12002F
:086B98000201B36BB26B010EA8
:106BA00000D012000201B251010B006E016A0050C8
:106BB000011007E0006A016A00C0F3FF01C0F4FFA2
:106BC000A1D00401180E746F5E0E756FB9C2E9FF93
:106BD000BAC2EAFFEF50006E016A0050011007E1EF
:106BE0000068016800C0F3FF01C0F4FF8BD0B9C298
:106BF000E6FFBAC2E6FFAFEC3BF0E552E552F3CF59
:106C0000B9F2F4CFBAF20F0EE66EE66A74C400F081
:106C100075C401F0026A00C0E6FF01C0E6FF02C0D1
:106C2000E6FF650EE66E040EE66E53EC3BF0F56E85
:106C3000070EE15EF55004016551006E016A0050D7
:106C4000011040E1B9C2E6FFBAC2E6FF76EC3BF0C4
:106C5000E552E552F3CF76F404017651006E016AF5
:106C60000150000AE8AE02D0013405D00C0ED880E5
:106C70000054000E015402E20C0E766F7651E66E5F
:106C8000E66A680EE66E040EE66EB9C2E6FFBAC2A8
:106C9000E6FF84EC3BF0F56E060EE15EF550000970
:106CA0000BE166C4B6F267C4B7F20201B32B66C447
:106CB000F3FF67C4F4FF26D00F0E04017427000E03
:106CC00075231FD06551006E016A040E001801E1A2
:106CD000015010E1661D01E1671D05E066C474F412
:106CE00067C475F40ED00068016800C0F3FF01C0EE
:106CF000F4FF08D00068016800C0F3FF01C0F4FF92
:106D000001D081D712000201B86BB291B351006E6D
:106D1000016A0050011001E0B3071200B4C2F6FF8F
:106D2000B5C2F7FF0800F5500401656F0201B42BEE
:106D3000000EB52304016551006E016A030E0018B0
:106D400001E101500CE1B4C2F6FFB5C2F7FF080043
:106D5000F550656F0201B42B000EB5230BD06551C1
:106D6000006E016A040E001801E1015003E1020106
:106D7000B469B5690401655100D012000201B28105
:106D8000200E006E016A00C0F3FF01C0F4FF00D0C6
:106D90001200010E00D01200B4C2F3FFB5C2F4FF1E
:106DA00000D01200B6C2B4F2B7C2B5F20401006B53
:106DB000016B040100C400F001C401F0002B000EBF
:106DC00001230201BC51001802E1BD51011802E08B
:106DD000A5DFEFD7B4C2F3FFB5C2F4FF00D01200B5
:106DE000FF0EE3CFEAFFE552FF0EE3CFE9FFE552E6
:106DF000E66AE66AD9CFE6FFDACFE6FFFC0EE124C9
:106E0000D96EFF0EE220DA6EE66AE66AE66A200EC6
:106E1000EF5C06E0090EEF5C03E0EF6603D03FD0C5
:106E2000EE50F5D72D0EEF5C03E1FF0EE32A03D001
:106E30002B0EEF5C01E1EE502F0EEF6424D03A0EE2
:106E4000EF6021D0D890F90EE336FA0EE336FD0E4E
:106E5000DECFE3FFFE0EDDCFE3FFD890F90EE33681
:106E6000FA0EE336D890F90EE336FA0EE336FD0E4D
:106E7000E350DE26FE0EE350DD22300EEE5CDE2611
:106E8000000EDD22D9D7FF0EE3CFE8FFE85207E07E
:106E9000F90EE31EE32AFA0ED8B4E306E31EE55228
:106EA000E552E552FF0EE3CFDAFFE552FF0EE3CFE6
:106EB000D9FFE552E1CFE9FFE2CFEAFFED52ED5213
:106EC000EECFF3FFEFCFF4FF1200D9CFE6FFDACF1A
:106ED000E6FFFA0EE3CFD9FFFB0EE3CFDAFFFD0E9C
:106EE000E35209E72D0EDE6EFC0EE31EE32AFD0ED3
:106EF000D8B4E306E31EE652E652E652FD0EE12464
:106F0000E76EFF0EE220E46EE652F70EE3CFE6FFF7
:106F1000F70EE3CFE6FFD5EC37F0F90EE124E96E8A
:106F2000FF0EE220EA6EC5EC37F00AE1C2EC37F062
:106F300009E1C5EC37F008E1C2EC37F007E108D011
:106F4000D0EC37F0CBEC37F0D0EC37F0CBEC37F0BF
:106F5000D0EC37F0DE6AF90EE126FF0EE222FF0EDA
:106F6000E3CFDAFFE552FF0EE3CFD9FFE552FC0E87
:106F7000E124E96EFF0EE220EA6EEECFF3FFEFCFE1
:106F8000F4FF1200EF380F0B1200EF500F0B02E16D
:106F9000EE52D8841200EF380F0B300FDE6E120065
:106FA000EE500F0B300FDE6E1200FC0EE3CFE9FF48
:106FB000FD0EE3CFEAFF100EE66EEE6AEE6AEF6AB0
:106FC000D890FD0EE336FE0EE336ED36ED36EF36A5
:106FD000FF0EE30609E0F6EC37F0EE52F6EC37F080
:106FE000EE52F6EC37F0EDD7E56E1200030EEF240B
:0E6FF000E8B6EF6E300EEF24E8BEEF6E000C38
:026FFE00C8C207
:107000009FF4C9C2A0F40401A051A16F9F51A06FC9
:10701000A1519F6F9FC4F3FFA0C4F4FF00D01200E2
:10702000D9CFE6FFE1CFD9FFCAC28CF4CBC28DF431
:10703000CCC28EF4CDC28FF404018C0E906F040E7E
:10704000916F90C4E9FF91C4EAFF030EE926000E98
:10705000EA22EF508B6F90C4E9FF91C4EAFFEF5032
:10706000E66E90C4E9FF91C4EAFF030EE926000E24
:10707000EA22E552E750EF6E8B51E66E90C4E9FFCD
:1070800091C4EAFFE552E750EF6E90C4E9FF91C466
:10709000EAFF020EE926000EEA22EF508B6F90C441
:1070A000E9FF91C4EAFF010EE926000EEA22EF5043
:1070B000E66E90C4E9FF91C4EAFF020EE926000ED5
:1070C000EA22E552E750EF6E8B51E66E90C4E9FF7D
:1070D00091C4EAFF010EE926000EEA22E552E750CC
:1070E000EF6E8CC41AF08DC41BF08EC41CF08FC4DC
:1070F0001DF000D0E552E7CFD9FF12000401A76BC5
:10710000A86BA96BAA6BD0C29FF4D1C2A0F4D8908F
:10711000A0339F33CEC2A1F4CFC2A2F49FC400F02B
:10712000A0C401F09F07000EA05B0050011018E002
:10713000A1C4E9FFA2C4EAFF020EA127000EA22308
:10714000EECF00F0EFCF01F0000100510401A727BE
:10715000000101510401A823000EA923AA23DED7B0
:107160000201D051010B16E0A1C4E9FFA2C4EAFF5D
:10717000EF50006E016A026A036A01AE02D0026833
:10718000036800500401A7270150A8230250A92337
:107190000350AA23A7C4A3F4A8C4A4F4A9C4A5F4C3
:1071A000AAC4A6F4A5C49FF4A6C4A0F40401A551E2
:1071B000A61123E0A96BAA6BA7C400F0A8C401F034
:1071C000026A036A9FC404F0A0C405F0066A076A55
:1071D00000500424A76F01500520A86F025006201C
:1071E000A96F03500720AA6FA7C4A3F4A8C4A4F4EE
:1071F000A9C4A5F4AAC4A6F4D5D7A7C400F0A8C40E
:1072000001F0001E011E00C0F3FF01C0F4FF00D01A
:0272100012006A
:0E721200F00E83160F0E9512959A9598929A8B
:10722000839A8398809A2EEC1DF0F00E95168316A3
:107230008382808A3AEC1DF0809A34EC1DF0F00EC7
:1072400083168382808A3AEC1DF0809A3AEC1DF016
:10725000F00E83168382808A3AEC1DF0809A0F0E1E
:1072600095120201280EDA6F1AD80201280EDA6F81
:1072700016D80201080EDA6F12D802010C0EDA6F6E
:107280000ED80201010EDA6F0AD80201130EDA6F6E
:1072900006D80201800EDA6F02D800D012002CD876
:1072A000000901E0FCD7959A9598F00E9516831683
:1072B0000201DA51006E016A040ED89001320032E8
:1072C000E804FBE100508312839A83983AEC1DF0A6
:1072D000808A3AEC1DF0809AF00E83160F0E0201A0
:1072E000DA1583123AEC1DF0808A3AEC1DF0809A90
:1072F0000F0E951200D01200838A8398959A959864
:107300003AEC1DF0808A3AEC1DF08350006E016A61
:107310000050080B0BE0809A3AEC1DF0808A3AECA2
:107320001DF0809A839A010E0BD00AD0809A3AEC15
:107330001DF0808A3AEC1DF0809A839A000E00D0EE
:107340001200DBC2E9FFDCC2EAFFEFCF00F0016A06
:1073500000BE016800C022F400500DE022C400F01D
:10736000016A00BE016800C0DFF222D80201DB2BF7
:10737000000EDC23E6D71200DDC2F6FFDEC2F7FF07
:107380000800F5CF00F0016A00BE016800C022F4D9
:1073900000500DE022C400F0016A00BE016800C088
:1073A000DFF206D80201DD2B000EDE23E5D7120046
:1073B000A3DF000901E0FCD7959A9598F00E951689
:1073C0008316DFC200F0016A00BE0168040ED89087
:1073D00001320032E804FBE10F0E001483128388AF
:1073E000839A3AEC1DF0808A3AEC1DF0809AF00EF8
:1073F0008316DFC200F0016A00BE01680F0E0014A0
:1074000083123AEC1DF0808A3AEC1DF0809A0F0E40
:06741000951200D01200ED
:0A7416004D70537461636B20322E39
:1074200032302E303400444843502F476C65616E33
:10743000696E672E2E2E00426F6172642053657450
:1074400075702E2E2E00202020202020202020208D
:1074500020202020202000434F4D4D414E44532EEC
:1074600043474900494E4445582E48544D000D0AA3
:107470000D0A0D4D434850537461636B2044656D94
:107480006F204170706C69636174696F6E20763132
:107490002E3120284D70537461636B20322E3230B0
:1074A0002E30342C2053657020323420323030336B
:1074B000290D0A0D0A09313A204368616E6765207B
:1074C000426F6172642073657269616C206E756DC4
:1074D0006265722E0D0A09323A204368616E676553
:1074E0002064656661756C74204950206164647223
:1074F0006573732E0D0A09333A204368616E676520
:107500002064656661756C74206761746577617964
:1075100020616464726573732E0D0A09343A204346
:1075200068616E67652064656661756C742073754B
:10753000626E6574206D61736B2E0D0A09353A20F9
:10754000456E61626C6520444843502026204950B6
:1075500020476C65616E696E672E0D0A09363A2008
:1075600044697361626C6520444843502026204979
:107570005020476C65616E696E672E0D0A09373AB7
:1075800020446F776E6C6F6164204D5046532069C4
:107590006D6167652E0D0A09383A205361766520C2
:1075A0002620517569742E0D0A0D0A456E74657298
:1075B0002061206D656E752063686F6963652028A2
:1075C000312D38293A20000D0A496E76616C6964C4
:1075D00020696E70757420726563656976656420D4
:1075E0002D20496E7075742069676E6F7265642E08
:1075F0000D0A507265737320616E79206B65792076
:10760000746F20636F6E74696E75652E2E2E0D0A71
:017610000079
:0E761200FB0EE3CFF6FFFC0EE3CFF7FFFD0EFD
:10762000E3CFF8FFFE0EE3CFE9FFFF0EE3CFEAFF63
:10763000F90EE35003E1FA0EE35009E0F90EE30618
:1076400002E2FA0EE3060900F550EE5CF1E01200EA
:10765000D9CFE6FFDACFE6FFFA0EE3CFD9FFFB0E74
:10766000E3CFDAFFFC0EE3CFE9FFFD0EE3CFEAFF45
:10767000E9CFF3FFEACFF4FFF80EE35003E1F90E90
:10768000E35008E0F80EE30602E2F90EE306DECF6F
:10769000EEFFF2D7FF0EE3CFDAFFE552FF0EE3CFA6
:1076A000D9FFE5521200FB0EE3CFF6FFFC0EE3CF4D
:1076B000F7FFFD0EE3CFF8FFFE0EE3CFE9FFFF0E6D
:1076C000E3CFEAFFE9CFF3FFEACFF4FFF90EE3508F
:1076D00003E1FA0EE35009E0F90EE30602E2FA0EC6
:1076E000E3060900F5CFEEFFF1D71200FE0EE3CF5F
:1076F000E9FFFF0EE3CFEAFFF36AF46AEE5203E01C
:10770000F34AF42AFBD71200D9CFE6FFDACFE6FF1F
:10771000FA0EE3CFD9FFFB0EE3CFDAFFFC0EE3CF87
:10772000E9FFFD0EE3CFEAFFF80EE35003E1F90EA7
:10773000E3500AE0F80EE30602E2F90EE306DE503B
:10774000EF5C02E1EE66F0D7F36EFF0EE3CFDAFFF7
:10775000E552FF0EE3CFD9FFE552F3501200FE0EC3
:10776000E3CFE9FFFF0EE3CFEAFFE9CFF3FFEACF74
:10777000F4FF610EEF5C05E67B0EEF5C02E7DF0EC7
:08778000EF16EE52F6E11200D3
:08778800485454502F312E30FB
:1077900020353033200D0A0D0A5365727669636512
:1077A00020556E617661696C61626C650D0A000D31
:1077B0000A0D0A00485454502F312E3020323030F8
:1077C000204F4B0D0A436F6E74656E742D74797083
:1077D000653A2000485454502F312E302034303434
:1077E000204E6F7420666F756E640D0A0D0A4E6F21
:1077F0007420666F756E642E0D0A000D0A4E6F7749
:107800002072756E6E696E67206170706C6963615D
:1078100074696F6E2E2E2E000D0A526561647920F8
:10782000746F20646F776E6C6F6164204D504653A7
:1078300020696D616765202D2055736520586D6F37
:1078400064656D2070726F746F636F6C2E0D0A002B
:107850000D0A44484350202620495020476C65615A
:107860006E696E672064697361626C65642E0D0ACF
:10787000000D0A44484350202620495020476C659B
:10788000616E696E6720656E61626C65642E0D0ABB
:10789000000D0A44656661756C74205375626E65EF
:1078A00074204D61736B2028000D0A446566617574
:1078B0006C742047617465776179204164647265F6
:1078C00073732028000D0A44656661756C74204945
:1078D0005020416464726573732028000D0A53655B
:0E78E0007269616C204E756D62657220280021
:0278EE005458EC
:1078F000540048544D0047494600434749004A5008
:107900004700434C410057415600746578742F700E
:107910006C61696E000000000000000000007465EA
:1079200078742F68746D6C00000000000000000087
:107930000000696D6167652F6769660000000000DF
:10794000000000000000746578742F68746D6C008E
:1079500000000000000000000000696D6167652FF5
:107960006A706567000000000000000000006170A0
:10797000706C69636174696F6E2F6A6176612D76D0
:107980006D00617564696F2F782D776176650000F1
:10799000000000000000485454502F312E30203297
:1079A0003030204F4B0D0A436F6E74656E742D742A
:1079B0007970653A20000D0A0D0A004745540049C8
:0979C0004E4445582E48544D0078
:0679CA002A0EF66E000E0D
:1079D000F76E000EF86E02010900F550C36F090042
:1079E000F550C46F03E1C36701D03DD00900F550E5
:1079F000BE6F0900F550BF6F0900F550C06F090058
:107A00000900F550E96E0900F550EA6E0900090019
:107A10000900F550C16F0900F550C26F0900090057
:107A2000F6CFC5F2F7CFC6F2F8CFC7F2BEC2F6FF67
:107A3000BFC2F7FFC0C2F8FF0201C15302E1C25347
:107A400007E00900F550EE6EC107F8E2C207F9D76A
:107A5000C5C2F6FFC6C2F7FFC7C2F8FF0201C307DF
:087A6000000EC45BBFD7120049
:087A68000101FF6B1200FFC1D8
:107A700000F0016A00BE0168005001E1015001E020
:107A80001BD00001260EF96F040EFA6F00011C0EC8
:107A9000F76F040EF86F32EC2FF0000901E11ED0F1
:107AA00004012651006E016A0050011002E116D057
:107AB00003D00101010EFF6F84EC23F000090CE0FC
:107AC0000001FD6B00011C0EFB6F040EFC6F01EC4E
:107AD00030F00101FF6B02D0000E02D0010E00D089
:027AE000120092
:0E7AE2003C0ED66ED768070ED56ED58EF28498
:107AF000F28A1200D9CFE6FFE1CFD9FFE0C21AF037
:107B0000E1C21BF0E2C21CF0E3C21DF000D0E5525E
:107B1000E7CFD9FF1200F250040B01E0010E006E16
:107B2000016A005001100AE0D7683C0ED66E0201CF
:0E7B3000E02B000EE123E223E323F294120087
:027B3E00FF0E38
:107B4000E350216E480E01D04C0EE76EE72EFED7B3
:0E7B5000E76AE72EFED7212EF7D700001200BD
:027B5E0015EE22
:107B600000F025EE00F0F86A209CA68EA69CE5ECBD
:0A7B70003CF061EC17F0FDD71200A5
:067B7A00FF0EE350E84E8F
:107B80001200000000D000D000D0E82EFAD712007A
:107B90000000000000DC78C578A9789178717850F1
:057BA000781878FB7766
:027BA5000000DE
:087BA700D477B477AF7788773B
:017BAF0000D5
:037BB000FF0000D3
:047BB30000000000CE
:020000040030CA
:08000000FFFAFFFEFFFEFBFF0B
:00000001FF
